:020000040800F2
:20000000182F0020A12C0008092C00080B2C00080000000000000000000000000000000028
:200020000000000000000000000000000D2C000800000000000000000F2C0008112C0008F7
:200040001B1500081B1500081B1500081B1500081B1500081B1500081B1500081B150008E0
:200060001B1500081B1500081B1500081B1500081B1500081B1500081B1500081B150008C0
:200080001B1500081B1500081B1500081B1500081B1500081B1500081B1500081B150008A0
:2000A0001B1500081B1500081B1500081B1500081B1500081B1500081B1500081D2C000867
:2000C000FFFFFFFFFFFFFFFFFFFFFFFFFFFFFFFFFFFFFFFFFFFFFFFFFFFFFFFFFFFFFFFF40
:2000E000FFFFFFFFFFFFFFFFFFFFFFFFFFFFFFFFFFFFFFFFFFFFFFFFFFFFFFFFFFFFFFFF20
:20010000000000000000000000000000000000004A2D4C696E6B204F422D53544D3332465D
:200120003037322D436F727465784D20636F6D70696C6564204D6172202038203230313629
:200140002031313A31353A35342000436F7079726967687420323030332D323031342053B5
:2001600045474745523A207777772E7365676765722E636F6D20000000000000000000001E
:20018000FFFFFFFFFFFFFFFFFFFFFFFFFFFFFFFFFFFFFFFFFFFFFFFFFFFFFFFFFFFFFFFF7F
:2001A000FFFFFFFFFFFFFFFFFFFFFFFFFFFFFFFFFFFFFFFFFFFFFFFFFFFFFFFFFFFFFFFF5F
:2001C000FFFFFFFFFFFFFFFFFFFFFFFFFFFFFFFFFFFFFFFFFFFFFFFFFFFFFFFFFFFFFFFF3F
:2001E000FFFFFFFFFFFFFFFFFFFFFFFFFFFFFFFFFFFFFFFFFFFFFFFFFFFFFFFFFFFFFFFF1F
:20020000F8B5040000250027002C01D10120F2BDF420400026187078002803D135702000D8
:2002200000F0CCFE032070700CE01C21794361182922885428228F542B228D544D638D6381
:20024000CD637F1C012061688F42EED300210CE01C224A43A21884235B00D2185570117093
:20026000D570D56015615561491C62689142EFD322684023D0522268D55222684423D5523C
:2002800022685023D552BF21090222684023D1522421655470700020F2BD00685821415A16
:2002A000802212020A43582142520020704738B5040020684421405A000402D5200000F0F4
:2002C000D1FC20684421415A49050CD54421415A334A0A4044214252200000F0B1FE0021FA
:2002E000200000F06BF82068010040318A88520403D58A882B4B13408B808A88920403D5EB
:200300008A88294B13408B8080256D018A882A4211D04022805A254A02400A80BD20000231
:200320000880200000F0A8FE20684421415A204A0A40442142522068010040318A88120527
:2003400013D58A881B4B13408B804022825A082313430B804022805A042202430A80888854
:20036000284202D1200000F077FE20684421415A890508D54421415A0F4A0A40442142522C
:20038000200000F056FE20684421415AC90505D54421415AB44A0A404421425231BD00009A
:2003A000FFFB0000FFBF0000FFDF0000FBFF0000FFEF0000FFF70000FFFD0000F422520065
:2003C00082181378012B01D102207047012313700B0004D1802100684C23C15201E02423E7
:2003E000C154002010707047F1B581B07F247F250D401C26754340190D0601D5283002E0B0
:2004000084256D0040190C400470C90941701100C260C370019AF4235B00D25C012A01D18C
:200420000220F6BD0122019BF42464001A558F4AC378002B05D0022B0DD01ED3032B13D01D
:2004400026E0019B1B680478A4001B191C8822408024A4001AE0019B1B680478A4001B1968
:200460001C8822401A8013E0019B1B680478A4001B191C882240C02407E0019B1B6804780A
:20048000A4001B191C8822408024E40014431C800478019A1268A300D518754B2E88754FA8
:2004A000374027431F432F800678C024A401724D877A002F59D1F600009687886F4E3E4054
:2004C0004778002F1CD05021515A009C091989188024E40009190E800178890051180C8890
:2004E000660604D5634E2640B74C34430C8000788000101801880D40202169400B43B1E0DB
:200500005025555B009FED19AD185F09ED192E805025555B0678F600AD19AD18BE1CAD196C
:200520003F2908D34E09C90600D1761EB60280210902314304E04E08C90700D5761CB102F1
:2005400029800178890051180D886E0404D5494E2E409E4D35430D80007880001018018809
:200560009B4A0A40544023437CE0B10051180F88404E3E40974F37430F805021515A0678B0
:20058000F600891989188026F6008919C6883B4F37400F805021515A0678F6008919891833
:2005A0005E0989190689354F37400F800178890051184678002E2BD10E88770404D52D4F60
:2005C0003740824E3E430E800178890051180E88770604D5274F37407B4E3E430E80017830
:2005E000890051180F88234E3E40774F37430F800178890051180E88754F37407C401C435D
:200600000C8000788000101801880D402B4329E00C88660404D5174E26406C4C34430C8084
:200620000178890051180C88660604D5114E2640654C34430C800178890051180C880D4EA3
:200640002640624C34430C800178890051180C8825401D430D8000788000101801885C4AE3
:200660000A401343A9E00000FFFE00008F890000808000008F8F0000BF8F0000FEFF0000D3
:20068000F1B581B07F227F230B401C246343C0180B0601D5283002E084235B00C0180A40F2
:2006A0000270C90941700199F4225200895C012901D10220F6BD0121019AF4235B00D15439
:2006C00001990968027892008A1800924678404A8025ED018D4B8E4C877A002F16D1002EFD
:2006E0000AD0009A1288550637D58A4D1540364A2A43009D2A8030E0009C24882C4256D039
:20070000844D2540314C2C43009D4FE0002E009E368829D12E4205D07E4D35402B4E2E43F8
:20072000009D2E800578AD004D192E88770604D5784F3740244E3E432E800578AD004D1963
:200740002F88744E3E40204F37432F800578AD004D192E8832401A432A8000788000081833
:2007600001880C40234328E02E4205D0694D3540164E2E43009D2E800578AD004D192E8860
:20078000770604D5634F37400F4E3E432E800578AD004D192F885F4E3E400C4F37432F8058
:2007A0000578AD004D192E8834401C432C8000788000081801880A401343038000200199F6
:2007C000F42252008854F6BDC080000080C000008FBF000080810000F1B582B07F20029C3E
:2007E0007F250D401C267543641984256D006419226163610022A26162700840207002984E
:20080000F4214900401801900078012801D10220FEBD012301990B706069E268824201D25E
:20082000801A01E0020000206061500851091340009380231B02A57A002D2DD06578002DAF
:200840001AD1029D2D685026AE5B2778FF00F61975199F4EAD193F2A06D30E00D70600D10E
:20086000761EB6021E4305E00600009F002F00D0761CB6022E800CE0012D27D1029D2D6804
:200880005026AE5B2778FF00F6197519904EAD192A806578002D19D1029D2D685026AE5BA9
:2008A0002778FF00F6197519A94EAD193F2A06D3D00600D1491E880203432B8014E00099E8
:2008C000002900D0401C800228800DE0607801280AD1029800685021415A2378DB00C9186B
:2008E00008189B4940180280029800682178890040180188084A0A40C02189015140034A30
:200900000A430280002001990870FEBD80800000BF8F00008F8F00008FBF00004906490EBB
:200920001C225143401890214900405880B27047F1B584B07F20049C7F250D401C2675430E
:20094000651928352A616B610022AA6101226A70084028700498F421490040180190007800
:20096000012801D10220B1E001990A706869EC68844201D2001B01E0040000206861049872
:2009800000680090A87A002811D1A3B2AA882969009800F041F9049800685021415A2A78A6
:2009A000D200891808184A49401804807EE060096B782E78224002921F21009AB700D25D2F
:2009C00052062AD5624A002B1AD1009B5027DB5BF6009B19009E9B199A183F2C08D3214061
:2009E00000D1401E8002802109020143118012E060080299002900D0401C800210800AE07F
:200A0000012B08D100985021405AF100401800994018801804802A892AE0002B1BD1009A6A
:200A20005023D25AF300D218009BD218284BD2183F2C08D3214000D1401E80028021090254
:200A40000143118013E060080299002900D0401C800210800BE0012B09D100985021405AD0
:200A6000F100401800994018194940180480EA88A3B22969009800F0CFF869785F480029A5
:200A800008D1049909682A78920089180A8810405B4A09E0012909D1049909682A789200E4
:200AA00089180A881040574A02430A80049800682978890040180188534A0A40302151406B
:200AC000524A0A43028000200199087005B0F0BD02040000B8B5F422520083181A78012AE4
:200AE00001D10220B2BD01251D707F220C0606D57F240C401C277C430419283405E01C24C3
:200B00004C43041984277F00E419A5700A402270C909617001683D48150004D10A883C4C7C
:200B20001440C2080DE0920089186278002A0A8803D0354C1440102203E0364C14408022AC
:200B4000520162401043088000201870B2BD000006040000F8B57F250A0606D57F220A407D
:200B60001C235A438218283205E01C224A43821884235B00D218002393700D401570C909A5
:200B80005170F4214900415C012901D10220F2BD0121F424640001550468117889006118E1
:200BA00000911A49154D5678002E009E36880ED0770604D53540124E2E43009D2E80127838
:200BC0009200A2181488104D254030240EE0770404D535400B4E2E43009D2E80127892002F
:200BE000A21814880B4D2540C024A4016C4021431180F421490043540020F2BD8F8F0000D6
:200C0000C080000080C00000BF8F000080800000BFBF00008FBF000010B510188022D200D9
:200C200080185B1C5A0807E00B784C7824021C430480801C891C521EF6D110BD18B51018D2
:200C40008022D20080185A0806E00488801C0C70240A4C70891C521EF7D1DA0701D5008896
:200C6000087011BDFEB500216A461180CA4F040028E00188C94A0A40028020685021415AF8
:200C80002822A25CD20089180818F91C4018008838402064A16B0818A0630021200000F028
:200CA000BDF92420205C00280CD0E06B002809D12420205C8021014320684C2281520020DF
:200CC0002421605420684421415A6A461180090400D45EE1694609880907090F00D087E093
:200CE00069460988C906C4D501000A886B461A801B881B0521D55022825A84235B00E35C26
:200D0000DB00D2185118A64A89180B883B408421490061188B618421490061188A88F62123
:200D200049006118FFF78AFF206801889D4A0A400280200000F05BF9C4E768460088000465
:200D4000C0D598481040088020685021415A84225200A25CD20089180918914A89180B8819
:200D60003B408421490061188B61002B16D08421490061188A888421490061180969FFF74C
:200D80005DFF842040002018006984214900611889694018842149006118086100212000B0
:200DA00000F02FF920685021415A08187C494018842149006118C9683F2908D34A09C9064D
:200DC00000D1521E920280210902114304E04A08C90700D5521C9102018020680188724A14
:200DE0000A40C02189015140704A0A43028069E78A000292821810886B4618801C23594360
:200E0000611801916946098809045BD565490140118001988421490046183378D9002068D9
:200E2000B57A002D0FD15023C35A591809185C4A891809883D000D402FD02B00B2883169F4
:200E4000FFF7FCFE29E09B00C35A5B040CD55023C35A59180918FA1C891809883D000D40AD
:200E600011D02B00F2880BE05023C35A591809184B4A891809883D000D4004D02B003289D4
:200E80003169FFF7DBFE20683178890040180188474A0A40474911430180B0694019B0618B
:200EA00031694A1932617369002B02D0F068854204D23178200000F0A4F803E031782000D3
:200EC000FFF78AFC6846008800065DD5019D28352068029940180188304A0A4002802B7840
:200EE000D80022681100AE7A002E0FD15023D25A10184018F91C401803883B40AB612ED0AD
:200F0000AA8829692068FFF787FE28E09B00D35C5B060BD55023D25A10184018F91C40186B
:200F200003883B40AB6110D0EA880AE05023D25A101840181A49401803883B40AB6104D0A3
:200F40002A8929692068FFF767FE20682978890040180188164A0A40174911430180297856
:200F600020685022825ACB00D2181018FA1C801800883840A8612A6912182A616B69002BC0
:200F800003D1200000F04AF89CE62000FFF7D0FC98E60020FEBD0000FF0300000F8F0000CE
:200FA000060400008F0F00008FBF0000808000008F8F0000C080000080C00000006892495A
:200FC000884200D0704780B5802000048F490A6802430A60096808400090009800220121C9
:200FE0001F2000F035F91F2000F036F901BD80B5F6214900411887229200805800F099F9F5
:2010000001BD80B51C224A4382188C235B00D25887239B00C05800F0B9F901BD80B51C2214
:201020004A438218926B87239B00C05800F0E3F901BD80B587218900405800F05CFA01BDA3
:2010400010B58721890044180121206801740020206800F01EFA10BD10B5040087208000B2
:20106000205800F038FAA069002804D06848016806220A43026010BD10B50400A06900281A
:2010800006D06348016806229143016000F07EFA87208000205800F027FA10BD10B501005E
:2010A0005C48872292008150121D8C1820605649016008214160022181600022C2600161B9
:2010C0008261C2610262FFF79BF8002804D0FF214031002000F0DCFA1823002200212068A4
:2010E00000F0D9FA582300228021206800F0D3FA982300228121206800F0CDFAD8230022CF
:201100000121206800F0C7FA90235B0000228121206800F0C0FAC0235B0000220121206866
:2011200000F0B9FA002010BD10B50024882189004058FFF7B2F8002804D0022801D10124AF
:2011400000E00224200010BD38B515001A0000242B008825AD004059FFF746F938E010B52C
:201160000024882292008058FFF78AFAE3E710B50024882292008058FFF7ACFCDBE710B5D1
:201180000024882292008058FFF7E4FCD3E781B08822920080584A06520E1C235A4380181E
:2011A000090601D52A2101E085214900405C01B0704710B50024882292008058FFF7FEF842
:2011C000B9E738B500248825AD004059FFF7B0FB002804D0022801D1012400E00224200087
:2011E00032BD38B500248825AD004059FFF7F4FAEEE780B5882292008058FFF78FFB02BDBB
:201200000548704700000000005C00401C10024010ED00E0DC060020FC08002018B5C2002E
:2012200018231340FF249C40E2438907090E9940002804D51C4B0007000F083800E01B4B78
:2012400080088000181803681A401143016011BD80B5FFF7E3FF01BD0121C006C00E8140CC
:2012600013480160704710B5401E80214904884201D3012010BD0F4C606003210020C043FC
:20128000FFF7CCFF0020A0600721216010BD09490428086803D1042202430A607047042283
:2012A00090430860704700001CED00E000E400E000E100E010E000E080B5C046C04601BDFF
:2012C00010B5002801D1022010BDFE235B00C3189C69002C01D000249C61002900D0596133
:2012E000012119700270FFF7D9FE002010BD02000020002903D085239B00D15070470220BC
:20130000704780B5FFF710FF002002BD10B50224852292008258002A04D012689047002888
:2013200000D10024200010BD80B5852292008258EFE038B50400822080002518280000F04C
:2013400079FBFA204000201801210160418B4160017DC806C00E03D002280BD005D30EE0DF
:201360002900200000F0B4F90EE02900200000F053FA09E02900200000F06BFA04E0802008
:2013800001402000FFF7F3FE002032BD38B504001000FA225200A3180A0021D11968032923
:2013A00027D18621490061184A680D68AA420AD2AB1A0B60934200D21A0092B20100200087
:2013C00000F08AFB15E0186A0169002904D0187A032801D120008847200000F081FB08E0C8
:2013E000186A8269002A04D0187A032801D120009047002032BDF8B505001000FA225200BD
:20140000AC180A003AD100262168022931D1E9692A6A00928A4207D28A1AEA6192B20100C6
:20142000280000F055FB11E0AF693800114600F06FFB002911D1009887420ED36068874274
:201440000BD20022280000F043FB66600023002200212800FFF7C5FE0BE0206AC168002963
:2014600004D0207A032801D128008847280000F043FB207B01280AD1267308E0206A42695F
:20148000002A04D0207A032801D1280090470020F2BD38B50500402300220021FFF754FE09
:2014A0004024882040002C504023002280212800FFF74AFE2C62FE2040002A180120107009
:2014C000D069002805D06968C9B22800926952689047002032BDFE214900401801784170DD
:2014E0000421017000207047FE2149004018417801700020704780B5FE21490041180A7846
:20150000032A04D18969C969002900D08847002002BD52689047002002BDFEE710B582B0B2
:2015200000F012FB00F032F853480168534A914202D1002101600BE0514CB821090220003F
:2015400000F01AFB002803D172B6200000F032FC002000F053F8002000F074F800F032FC2F
:20156000484800780328FBD1002000F079F8642000F040FC002000F073F80121684600F000
:2015800026FC6846007800F08BFBEDE710B598B020200B9001201390002414940BA800F09E
:2015A00039FC002800D0FEE70720009003200190029403940121684600F038FE002800D093
:2015C000FEE78020800204900A9404A800F030FF002800D0FEE700F001FFFA21890000F0A6
:2015E00097FAFFF740FE0420FFF751FE002200210020C043FFF72CFE18B010BD30B587B086
:2016000080218902204A13680B43136012681140009100991FA142008D5A019501210291CF
:201620000021039103210491184980000C1801A9206800F09DFF00222900206801F06AF853
:2016400007B030BD80B5002200E0000011A14300C95A0E4B8000185801F05CF801BD00004B
:2016600080B500BF0BA14200895A084A8000105801F058F801BD00000001002021433412A1
:2016800000480008B40600201410024000030020FEE70000010010B50C0606D54906490E59
:2016A0001C2461434018283005E01C244C430019842149004018002A03D10021817283806E
:2016C00004E001218172C380190C0181002010BDF8B504000F00FE20400025180020022697
:2016E0007978092951D802A2525C5200974400BF6D804D7D4D0A054D5D2A3900200000F030
:201700001BF985E0B88800283FD1F88800283CD16846B9784906490E01702878032834D05E
:20172000A970684601782000FFF743FD200000F0D7F968460078002801D02E7068E001200D
:20174000287065E07988334A1170117802291CDA0A002B78022B1DD0032B16D1002905D128
:201760002E7060602000FFF7DFFD4EE061688A424BD0C9B22000FFF7D7FD2648017861602E
:201780002000FFF7C3FD02283FD13900200000F065F93DE0002938D06260032028702000A7
:2017A000FFF7B4FD0228F0D02FE0F9880129ECD12978022904D00329E7D10122211D10E04C
:2017C000A0600122210008310BE02978891E0129DBD8E060A868002800D0E66002222100A9
:2017E0000C31200000F066F912E07888012805E02978891E0129C8D87988012908D1A8601F
:2018000039002000AA6992689047200000F068F90020F2BD140F002038B505000C00FE20EC
:2018200040002A18107803280ED1A088C0B202280ADA2800926992689047E088002806D191
:20184000280000F04DF902E0280000F007F9002032BD70B582B004000E00B188C9B2FE20E6
:2018600040002518307860220240202A05D131002000AA69926890475CE07F227F20084066
:201880007378002B2ED0012B11D0032B52D12878022812D0032849D17088002819D10029B2
:2018A00017D0802915D02000FFF761FC11E02A78022A02D0032A04D038E000293AD08029BA
:2018C00017E07288002A35D1002807D02000FFF756FC31002000AA6992689047200000F03B
:2018E000FFF827E02B78022B02D0032B06D01DE000281FD02000FFF73AFC1BE00A4010018E
:2019000020180A0602D50500143502E08222520085182000FFF73BFC002800D001202860F7
:2019200002222900200000F0C5F803E03100200000F094F8002076BD70B582B004000D0022
:201940006888842189006218010A012908D002291FD003292AD0062955D007295BD064E0AF
:201960006946207C1268126890476946098800290ED0E98800290BD06A4612888A4200D9A6
:201980000A0069460A800A880100200000F092F873BD51680226207C0028684603D1896A8D
:2019A00088474670E1E7C96A8847FAE7C0B205283BD801A1095C8F4404101C2834406946F0
:2019C000207C126852689047CFE76946207C126892689047C9E76946207C1268D26890478E
:2019E000C3E76946207C126812699047BDE76946207C126852699047B7E76946207C1268C8
:201A000092699047B1E7207C00280ED168465168496B8847A9E7207C002806D1684651683D
:201A2000096B8847072141709FE72900200000F015F873BD0A7802704A7842708A78CB78E1
:201A40001B02D21842800A794B791B02D21882808A79C97909025118C180704710B50400F3
:201A60008021FFF784FB00212000FFF780FB10BD002800D1704770B504000023002501E0CF
:201A80006D1C641C2678002EFAD12D06EC0DA41C148012880A7003224A70022206E0D2B2A5
:201AA0008C54401C521CD2B28B54521C0478002CF5D170BD10B513000222FA24640002513F
:201AC0008361C3610A000021FFF77BFB002010BD80B513000A000AE080B513000A0012E0FA
:201AE00080B50421FA2252008150002300220021FFF767FB002002BD80B50521FA225200E7
:201B00008150002300220021FFF76BFB002002BD094214D088420FD30122030C01D1000470
:201B20001204002300185B418B4200D35B1A5241F8D319001000704701000020704708B5D0
:201B4000C046C04608BD000080B50648016810220A430260002000F0F5FD00F005FE0020D2
:201B600002BD00000020024008B4024B9C4608BC6047C046D9030020F8B502000B009C1E78
:201B800000920027002511E0060008E0565D7E40F6B208217008F607F6D5714E4640491E5A
:201BA000F8D1380A37004740BFB26D1CA542EDD3D018801E0088874202D00020C043F2BD40
:201BC0000020F2BD00000000F0B583B000200190012101A800F003F90221684600F0F7F846
:201BE000684600885F4988420EDB022100A8801C00F0EDF8684600885B4901406846408887
:201C00008003084369460880584D80218900280000F0DDF81C2200BF5EA1882040002818DF
:201C200000F0C2FD0190002800D0FEE7504FFE0C0123320029003800FFF796FF0123320046
:201C4000A9184C48FFF790FF02240BE03100280000F0BDF80123320029002002C019FFF72B
:201C600083FF641C68460088000A8442EEDB684601883800FFF780FF002800D00120019005
:201C8000012101A800F0ABF8642000F0B3F8BFF34F8F394839490860BFF34F8F00BFFDE799
:201CA00000B589B080214900884202DB0020C0431CE0002201280ED0042819D0052825D026
:201CC000062828D0072829D0E62839D0ED2839D0F02841D043E0702000900221684600F054
:201CE0007EF80099264800F07AF8002009B000BD244800900221684600F071F880200001A8
:201D000000900221684600F06AF8EEE70221684600F05DF8E9E7FFF757FFE6E7684600216D
:201D200000230AC06846E42101700C21417001218170C270017142718171C1710821E2E734
:201D40001148D0E76846202100F05AFD0F4800900F4801902021D5E700920421D2E7FEE71C
:201D60000884000001800000FC3F0000100B002000480008004900080400FA050CED00E063
:201D800010010008E32E000000020020090060880C2800004A2D4C696E6B204F422D535448
:201DA0004D3332463037322D436F727465784D2000000000016881F308884068002282F3D7
:201DC0001488004780B500F01DFD002002BD80B50A000100064800F0A9FD002002BD80B5CA
:201DE0000A000100024800F0EBFD002002BD0000B804002031B500F001FE0400009D002065
:201E0000C043854200D06D1C00F0F8FD001BA842FAD331BDF8B504008B4D2078C00700D43E
:201E200027E18026B60268680C21014004290BD068680C21014008290ED16868C0214902AC
:201E400001407008814207D12868064032D06068002821D10120F2BD6168012908D07B4816
:201E600000290AD0052908D12868710001432960286871080143296006E02968744A0A4035
:201E80002A60296808402860606800280DD000F0B5FD07002868304000D0EAE000F0AEFDAC
:201EA000C01B6528F6D30320F2BD00F0A7FD07002868304000D1DCE000F0A0FDC01B652802
:201EC000F6D3F0E700F09AFDC01B022800D801E1E9E7E068002828680FD00121014329607E
:201EE00000F08CFD07002868304000D0DDE000F085FDC01B0228F6D9D5E70121884328605E
:201F000000F07CFD07002868304000D1D4E000F075FDC01B0228F6D9C5E701218843686233
:201F200000F06CFD0700686A304000D1D6E000F065FDC01B0228F6D9B5E7002801D1286A2A
:201F40000AE00528286A07D1042101432962286A01210143296206E0012188432862286A9A
:201F6000042188432862A06800280ED000F046FD0090286A304000D0DDE000F03FFD0099C2
:201F8000401AA9498842F4D38DE700F037FD0090286A304000D1CEE000F030FD0099401AAB
:201FA000A1498842F4D37EE700F028FDC01B022800D8D8E077E700F021FDC01B022800D84E
:201FC0000EE170E70421C9438842686B03D1042188436863CBE0042101436963686B012189
:201FE0008843686300F00AFD0700686B304000D1C4E000F003FDC01B0228F6D953E7206A0D
:020000040800F2
:202000000028686B0FD0F1030143696300F0F6FC0600686BC00300D5CDE000F0EFFC801B6C
:202020000228F6D93FE70A490140696300F0E6FC0600686BC00300D4BDE000F0DFFC801BDC
:202040000228F6D92FE700BF00100240FFFFFBFFFFFFFEFF0140296000F0D0FC0400286853
:20206000304000D1DEE000F0C9FC001B0228F6D919E70226206830401ED068680C2101404C
:202080000CD068680C210140082905D16868C02149020140B003814200D01AE7286830409B
:2020A00003D0E068012800D0D4E62868F82188432169C90001432960207800070ED5E069F3
:2020C0000028686A00D128E701210143696200F095FC0700686A304000D1F3E620784007A2
:2020E0002FD50027F006E969014007D1E9690143E961E9690840009000980127A148006839
:20210000C00513D49F480068A90D01439D48016000F074FC00909B480068C00506D400F0BA
:202120006DFC0099401A6528F5D3BCE6A068012800D002E70BE7002F03D0E8699249014001
:20214000E9612078C00619D56069012800D039E7686B042101436963686B012101436963FA
:2021600000F04CFC0700686B304000D11CE7686BF8218843A169C900014369632078800651
:2021800019D568680C2101400C290DD068680C210140082906D16868C02149020140C0209E
:2021A0004002814200D02AE7686BC00303D5206A012800D04EE6606A002833D069680C2220
:2021C0000A40082A00D145E68026B60485490228286800D03EE70140296000F00FFC0700DE
:2021E0002868304000D0E6E6E86A0F218843216B0143E96268687C490140E06A0843A16A65
:2022000001436960286871080143296000F0F6FB04002868304005D100F0F0FB001B022800
:20222000F7D940E60020F2BD89130000F2B582B00127FF4301246D4D29682140029A9142BA
:2022400008D2296839400A432A6029682140029A914222D10190664E0220019909680140BC
:2022600006D07168F0229143019A92680A43726001990968214068D001994968012902D129
:202280003068800308E0022902D13068800103E0032903D1706BC00303D465E0326810409D
:2022A00062D07068032290430143716000F0A6FB0199496801290ED1009070680C2101404C
:2022C000042942D000F09AFB0099401A49498842F3D30320FEBD02290DD1009070680C21A9
:2022E0000140082931D000F089FB0099401A41498842F3D3EDE70329009037D170680C214D
:2023000001400C2921D000F079FB0099401A39498842F3D3DDE701980078400706D570681E
:20232000354901400198C0680843706000F02EF8324972681206120F895CC8403049086090
:20234000002000F0FFF90020FEBD0298296821408842E0D22868074002983843286028688E
:20236000044002988442D6D00120FEBD70680C210140EAD000F042FB0099401A1D498842E7
:20238000F4D3A6E700700040FFFFFFEFF0B51D490B681D481D4A0C241C40082C02D00C2C39
:2023A0001AD0F0BD0F2500BF19A49E0C2E40A45D1BA6896A0D40715DC0256D022E001E400E
:2023C00080277F02BE4203D02B40AB4200D11000FFF79EFB6043F0BD1000F0BD0848006875
:2023E00070470000FFFFFFFEFF7FC2FF002002400010024089130000FFF8FFFF542B000820
:20240000040300200410024000127A00006CDC0202030405060708090A0B0C0D0E0F1010D2
:202420000102030405060708090A0B0C0D0E0F10F0B583B0040002270125464E2068C0030A
:2024400058D50020019028073168014007D1316801433160316808400090009801953E482A
:202460000068C0051CD43C480068290201433A48016000F0C3FA009037480068C0050FD435
:2024800000F0BCFA0099401A6528F5D30320FEBD00F0B4FA0099401A304988421AD3F5E7D3
:2024A000C02080007168014017D062681040814213D071682A48084071682A040A43726042
:2024C0007168284A0A4072607060284005D000F095FA009070683840DAD0706820490140FD
:2024E0006068084370600198002803D030681E49014031602068054005D07069032188432A
:20250000A168014371612068074005D0706917490140E068084370612078800605D5706949
:20252000102188432169014371612068800305D5706980218843A1690143716120684005E8
:2025400005D57069402188436169014371610020FEBD00001C100240007000408913000027
:20256000FFFCFFFFFFFFFEFFFFFFFFEFFFFFFCFFFEB500232FE0052503E0654DA842FAD129
:2025800004256F463F78BD403543019E3560674D2E68E5432E404F68FF0300D52643634F74
:2025A0003E607E682E404F68BF0300D526435F4F7E60BE682E404F68FF0200D526435B4FB2
:2025C000BE60FE6835404E68B60202D52E0025003543FD605B1C0D682C00DC4000D195E01B
:2025E00001249C4002942C40F4D06D469E006E704D68022D01D0122D1AD1DD08AD00451916
:202600002E6A01966E4677781C263E406F463E70019EB4466E4636780F27B7406646BE43F0
:20262000B4460F696E463678B740664637432F6205686E465F00377003266F463F78BE405E
:20264000F74301973E462E400D79AD07AD0F6F463F78BD40354305604D68012D05D0022D93
:2026600003D0112D01D0122D11D18668019D3540CE686F463F78BE402E4386604568029E12
:20268000B5434E68F706FF0F9F402F434760C668019D35408E686F463F78BE402E43C66051
:2026A0004D68ED0096D5224D2D6801262E43204D2E602D68EE07F60F0196019D1D4D9E08A2
:2026C000B600AD1901952E680C256F46BC467F783D4067463D706D462D780F27AF40BE431E
:2026E0009025ED05A84201D100254AE7124DA84201D1012545E7114DA84201D1022540E74C
:202700000F4DA84200D038E703253AE7F7BD00000010004881B0002A01D0816100E081625E
:2027200001B0704742694A404261704700040140181002400800014000040048000800480E
:20274000000C004810B50400FFF748FEFA218900FFF7DEF9FEF787FD002221000020C043D0
:20276000FEF776FD002010BD80B501200D490A6802430A6009680840009000980022002113
:202780000420C043FEF764FD002200210120C043FEF75EFD002200210020C043FEF758FD55
:2027A00001BD00BF1810024010B402E0401C491C521E002A09D00B7804789C42F6D002D2E1
:2027C0000020C04302E0012000E0002010BC7047130030B414001500103902D310393CC0CD
:2027E000FCD2490700D30CC000D504C0890002D30280801C002900D5027030BC70470000F4
:202800000022E5E710B5074C002207492000FEF757FD06492000FEF76AFD2000FEF771FD89
:2028200010BD0000B8040020780300200803002038B5040084208000FEF7E2FC8621890011
:2028400061180860002801D1022032BD050080208000281800210171417101600121C1603E
:202860004023022281212000FEF76EFC4023022201212000FEF768FC40232A0001212000BF
:20288000FEF7AFFC002032BD10B504008121FEF766FC01212000FEF762FC862080002418D0
:2028A0002068002803D0C046C04600202060002010BD10B5020000200B7860241C40202C66
:2028C00003D01000FFF7CAF8022010BD29210180474870470021862292008058133A815408
:2028E00000207047002070470020704700207047002070470020704738B50C0086218900A5
:202900004158802292008D182100FEF772FC2860012C04D12879002801D1012028710020C2
:20292000E86032BD0A21018032487047F1B582B086239B00C058183BC518EB68002BFCD1D4
:2029400016000C0072B60121E96062B62979012920D172B62A680100200000F055F80220B3
:20296000287162B60020009010232A6801212000C046C0462868864204D172B60020E86026
:2029800062B6FEBD2868864200D2FEE72868361A2868241840270FE0402E00D237000120BB
:2029A000E860BBB2220001210298FEF71AFCE8680028FCD1F61BE419002EEDD10020FEBD5F
:2029C00010B582B013008622920082580A4C14192278002AFCD172B60122227062B69BB283
:2029E0000A008121FEF7EDFB20780028FCD116BD400300206C030020050200000148006844
:202A0000704700BF100F0020124207D08B0706D00B78491C0370401C521EF7D87047830737
:202A200006D00B78491C0370401C521EF9D1704770B4103A03D378C9103A78C0FBD25307EA
:202A400001D318C918C001D508C908C0D20704D30B880380891C801C002A01D50B7803707D
:202A600070BC7047122008800F487047042008800E48704710B50A0010A008E010B50A00BC
:202A80000B4C21000FA004E010B50A000FA0084C2100FEF7EDFF200010BD000010B50A009B
:202AA000034C21000CA0F4E794030020A8030020100D002010B50A000AA0E8E74A2D4C69EC
:202AC0006E6B0000534547474552000030303030303132333435360042554C4B20436F6ECD
:202AE0006669670042554C4B20696E7465726661636500001148016801220A430260416864
:202B00000F4A0A40426001680E4A0A40026001680D4A0A40026041680C4A0A404260C16A81
:202B20000F229143C162016B094A0A400263416B01229143416300218160704700100240AD
:202B40000CB8FF08FFFFF6FEFFFFFBFFFFFFC0FF2CFEFCFF000000000000000001020304D4
:202B60000607080970B401000123002413E00A68091D1A4202D04D466D1E52191460121DE5
:202B8000001F0428FAD21500860701D51480AD1C184000D02C700868091D0028E7D1080007
:202BA00070BC704730B501684118446862088A188368E4070DD54C461B190AE00C7864B2D1
:202BC000491C0D78491C1D705B1C002C05D5641CF9D19142F2D10C3030BD641EF1D5F8E76C
:202BE00010B5074979441831064C7C44163404E0081D0A68891888470100A142F8D110BDF9
:202C00003C000000580000007047FEE77047704780B500F00BF8FEF74FFB01BD80B5024872
:202C2000FDF745FB01BD0000DC06002002480168491C0160704700BF100F002029FFFFFF4C
:202C4000600A0000B80400200000000059FFFFFF6C000000DC030000000200200120C04644
:202C6000002801D0FFF7BCFF002000BF00BFFEF755FC00F000F880B500F002F801BD000001
:202C80000746384600F002F8FBE7000080B500BF00BF024A11001820ABBEFBE726000200E2
:202CA0000148804701480047F52A0008B12C000800BF00BF00BF00BFFFF7D0FF030C5287BF
:202CC00003E4FF0347444200F4FF0352444900F4FF07466C617368425000F8FF07466C61DE
:202CE0007368444C00F8FF064A466C61736800F7FF04524444490081FFF4FFFD005A480005
:202D0000127A003128000889280008B3280008E9280008E5280008D5280008F9280008EDE1
:202D2000280008F1280008F5280008CD280008CD280008CD2800082529000809022900019B
:202D40000102C0320904000002FFFF0006070581024000000705010240F200030A06000246
:202D6000FD00014001FD001F652A00086D2A00087D2A0008752A0008892A00089D2A0008E2
:202D8000B52A000812010002FD007E406613010100020102030100000403090408B4024BDB
:202DA0009C4608BC6047C046A9270008002142181268FF2A06D1091D802212019142F6D37C
:202DC0000120704700207047F7B582B0324C334820603348206014250127002B2ED00298CE
:202DE00040052BD102980090E60C0098FFF7DEFF002818D1E06802210143E16000982061F1
:202E0000E06840210143E160A0687E3840FCD1A068800601D52020A060A068284012D1E0E2
:202E20006802218843E0600098FFF7C0FF1D4836180098E10C40180090002ED6DC049A030E
:202E400099002007E0A5600020C04322E0E368BB43E360801C904212D2E3683B43E3600BB3
:202E60005A029E36183380A3683B40FCD1A3689B0601D52023A360A3682B40E7D0E2E7E066
:202E80006880230343E3600298FF1EF788FF002800D0FEE705B0F0BD0000042002402301A0
:202EA0006745AB89EFCD00F8FFFFFFFFFFFFFFFFFFFFFFFFFFFFFFFFFFFFFFFFFFFFFFFF96
:202EC000FFFFFFFFFFFFFFFFFFFFFFFFFFFFFFFFFFFFFFFFFFFFFFFFFFFFFFFFFFFFFFFF12
:202EE000FFFFFFFFFFFFFFFFFFFFFFFFFFFFFFFFFFFFFFFFFFFFFFFFFFFFFFFFFFFFFFFFF2
:202F0000FFFFFFFFFFFFFFFFFFFFFFFFFFFFFFFFFFFFFFFFFFFFFFFFFFFFFFFFFFFFFFFFD1
:202F2000FFFFFFFFFFFFFFFFFFFFFFFFFFFFFFFFFFFFFFFFFFFFFFFFFFFFFFFFFFFFFFFFB1
:203F200047444200FFFFFFFFFFFFFFFFFFFFFFFF52444900FFFFFFFFFFFFFFFFFFFFFFFFED
:203F4000466C617368425000FFFFFFFFFFFFFFFF466C617368444C00FFFFFFFFFFFFFFFF73
:203F60004A466C61736800FFFFFFFFFFFFFFFFFF5244444900FFFFFFFFFFFFFFFFFFFFFFFA
:203F8000FFFFFFFFFFFFFFFFFFFFFFFFFFFFFFFFFFFFFFFFFFFFFFFFFFFFFFFFFFFFFFFF41
:203FA000FFFFFFFFFFFFFFFFFFFFFFFFFFFFFFFFFFFFFFFFFFFFFFFFFFFFFFFFFFFFFFFF21
:203FC000FFFFFFFFFFFFFFFFFFFFFFFFFFFFFFFFFFFFFFFFFFFFFFFFFFFFFFFFFFFFFFFF01
:203FE000FFFFFFFFFFFFFFFFFFFFFFFFFFFFFFFFFFFFFFFFFFFFFFFFFFFFFFFFFFFFFFFFE1
:020000040800F2
:204000000001FFFFFFFFFFFFFFFFFFFFFFFFFFFFFFFFFFFFFFFFFFFFFFFFFFFFFFFFFFFFBD
:20402000FFFFFFFFFFFFFFFFFFFFFFFFFFFFFFFFFFFFFFFFFFFFFFFFFFFFFFFFFFFFFFFFA0
:20404000FFFFFFFFFFFFFFFFFFFFFFFFFFFFFFFFFFFFFFFFFFFFFFFFFFFFFFFFFFFFFFFF80
:20406000FFFFFFFFFFFFFFFFFFFFFFFFFFFFFFFFFFFFFFFFFFFFFFFFFFFFFFFFFFFFFFFF60
:20408000FFFFFFFFFFFFFFFFFFFFFFFFFFFFFFFFFFFFFFFFFFFFFFFFFFFFFFFFFFFFFFFF40
:20480000601D00201DFA00081B690008836B0008000000000000000000000000000000005A
:20482000000000000000000000000000339200080000000000000000957900083DF7000859
:20484000D7A600080BA900084FBB000893BF0008EFD00008B3D2000841F4000893F6000889
:2048600003FA00080FFA000841FA000843FA000845FA000847FA000849FA00084BFA000872
:204880004DFA00084FFA000851FA000853FA000855FA000857FA000859FA00085BFA000868
:2048A0005DFA00085FFA000861FA000861BD0008B9D5000863FA000865FA00084FAA00084C
:2048C000FFFFFFFFFFFFFFFFFFFFFFFFFFFFFFFFFFFFFFFFFFFFFFFFFFFFFFFFFFFFFFFFF8
:2048E000FFFFFFFFFFFFFFFFFFFFFFFFFFFFFFFFFFFFFFFFFFFFFFFFFFFFFFFFFFFFFFFFD8
:20490000000000000000000000000000000000004A2D4C696E6B204F422D53544D33324615
:204920003037322D436F727465784D20636F6D70696C6564205365702032362032303136C9
:204940002031303A30333A353600436F7079726967687420323030332D323031342053454A
:20496000474745523A207777772E7365676765722E636F6D0000000000000000000000003B
:20498000FFFFFFFFFFFFFFFFFFFFFFFFFFFFFFFFFFFFFFFFFFFFFFFFFFFFFFFFFFFFFFFF37
:2049A000FFFFFFFFFFFFFFFFFFFFFFFFFFFFFFFFFFFFFFFFFFFFFFFFFFFFFFFFFFFFFFFF17
:2049C000FFFFFFFFFFFFFFFFFFFFFFFFFFFFFFFFFFFFFFFFFFFFFFFFFFFFFFFFFFFFFFFFF7
:2049E000FFFFFFFFFFFFFFFFFFFFFFFFFFFFFFFFFFFFFFFFFFFFFFFFFFFFFFFFFFFFFFFFD7
:204A000008B4024B9C4608BC6047C046F505002038B4002B1FD10400503478300078002849
:204A200001D0636A17E0206A00280CD0C500E4696419083C2568AA4201D363680BE0083C39
:204A4000401EF7D107E0C0239B032068AB4A904201D1F0231B04CB600120087431BC704709
:204A6000F8B50E0004005034002332002100FFF7CFFF00220221200001F068FA0500207D5F
:204A80000106022001F0BCFA07003100052001F0B7FA38436168A94206D06560060029004E
:204AA000042001F0ADFA30430500207D000610210143022001F0A4FA010029430800F2BDD5
:204AC000F8B50E0004005034002332002100FFF79FFF00220221200001F038FA0500207D5F
:204AE0000106022001F08CFA07003100052001F087FA38436168A94206D065600400290050
:204B0000042001F07DFA2043002802D50020C043F2BD0020F2BDF8B50024BE4E356AC8358D
:204B20000021072001F0BAFA01276946072001F0B5FA0098C00C384003D1306A281AF4D595
:204B4000E4432000F2BDFCB583B007000E003C0050340A9DA80001D5012020762807000F8C
:204B600002902068654988420BD1207E002801D0012200E0039A029882403100380001F0DA
:204B800045FBFF231B042B40320021003800FFF73FFF0B98019002980090049B039A31009F
:204BA000200001F048F90021217605B0F0BDF6B583B007001E003C00503401250A9881007D
:204BC00000D525760107090F01910A46012191407A22BA5C002A36D0039AB24B9A4232D115
:204BE000042977D10499012974D1AF493800FFF737FF00281DD40021072001F04FFA69468E
:204C0000072001F04BFA70780002B17809040143F07800060843A54A02400098F021090334
:204C200001401143072001F0EBF9002804D501F0DDF90020C0435CE001F0C4F900210320CA
:204C400001F02CFA44E0039AB94B9A4242D1042940D1049901293DD1300001F02AFC00909F
:204C6000B3493800FFF72CFF0028E2D10099072001F0C6F90028DAD401F0A4F90098400751
:204C800022D5022001F025FE0021032001F006FA00281DD05F4E306A9621C90040180190ED
:204CA000A44F642001F015FE6946002001F0F6F9002804D1009838409F49884208D001989A
:204CC000316A401AEDD503E00021032001F0E6F901200EE0FF231B04034021003800FFF744
:204CE00097FE019800903300049A0399200001F0F4F80021217605B0F0BD0000FF00010E64
:204D0000F2B582B017001C000100503101916649FFF7A6FE002807D40021072001F0BEF937
:204D20006946072001F0BAF90298007801F0E8FD009D000202210143062001F061F9B64E96
:204D400035402900072001F05BF90198FFF7E3FE002810D4009D0021062001F09FF9390027
:204D6000062001F09BF92E403100072001F048F90198FFF7D0FE002808D40298401C0290A7
:204D80003F1D641ED0D1002003B0F0BD0020C043FAE7F2B582B017001C007A21415C0029A3
:204DA00004D00299FFF7ACFF06002FE03E49FFF757FE002802D50020C04328E002980178BF
:204DC000052001F01DF90021042001F067F900265A48056AC8356946042001F05FF9009829
:204DE000C00305D45548006A281AF4D5F6430DE00021062001F052F93900032001F04EF9C8
:204E00000298401C02903F1D641ED7D1300003B0F0BD0000B8010020F2B582B017001C000F
:204E20000100503101912049FFF71AFE002807D40021072001F032F96946072001F02EF992
:204E40000298007801F05CFD009D000203210143062001F0D5F8704E35402900072001F097
:204E6000CFF80198FFF757FE00280CD4009D3968062001F0C5F82E403100072001F0C0F8FE
:204E80000198FFF748FE002808D40298401C02903F1D641ED4D1002003B0F0BD0020C0438B
:204EA000FAE70000FCED00E0F0ED00E0FFFFF0FFF2B582B017001C007A21415C002904D05D
:204EC0000299FFF7A9FF06002EE09349FFF7C8FD002802D50020C04327E03968062001F00D
:204EE0008FF802980078802149020143052001F087F80021042001F0D1F800260F48056A69
:204F0000C8356946042001F0C9F80098C00305D40A48006A281AF4D5F64305E00298401C00
:204F200002903F1D641ED8D1300003B0F0BD00000CED00E0FF0F000077040000B80100208D
:204F4000F0B583B007003E00503600247249FFF787FD05007A20385C002825D0002D1ED4E6
:204F60000021042001F09AF8050001A9072001F095F80095050002A9072001F08FF8010030
:204F80002943009D29430D0009D40198800302D57A203C5404E002980403E40F00E0E44316
:204FA0007A20385C002833D10021042001F076F804002C4301A9042001F070F8204315D50C
:204FC0000020706054493800FFF74AFD05000021042001F063F804002C4301A9042001F007
:204FE0005DF8204302D50020C04312E0019800030BD54A49042001F003F80021042001F0B8
:205000004DF801A9042001F049F801988403E40F200003B0F0BD0000FFFFF7FFF1B582B0EC
:20502000044679346078002842D03B490298FFF717FD0021072001F031F86946072001F016
:205040002DF800980103C90F07D1C0218902014300910099072000F0D3FF0021072001F0E3
:205060001DF82F4F3D6AC83501A9072001F016F8002802D50026F64308E001980603F60F3C
:2050800002D1386A281AEFD501980090002E0CD1002060700098234901400091072000F084
:2050A000AFFF0021072000F0F9FF607800282ED119490298FFF704FD2078C000174D05431C
:2050C0002900072000F09CFF01F03CF8144F3E6AB61C01A9072000F0E1FF002802D5002033
:2050E000C04306E001998803C00F02D1396A711AEFD506002078002809D008208543290056
:20510000072000F07DFF0021072000F0C7FF00202070300003B0F0BDF0ED00E003005FA0FF
:20512000B8010020FFFFFCFFF0B58BB00400CA07D20F04928807C00F69460873206DCA4949
:20514000884218D1200001F087F8002802D50020C04387E1200001F079F8C4492000FFF7DD
:20516000AFFC002807D40021072000F049FF002801D100F027FF6846007B002873D06846AF
:2051800000210173BA492000FFF79AFC80202058883000680125284202D0A843019005E0D0
:2051A00000F0D0FF01A9032000F078FF01993031052000F025FF00F0C5FF01A9032000F057
:2051C0006DFF019800284ED00021C94388424AD0A8430190014610392000FFF771FC0021C3
:2051E000072000F05BFF06A9072000F057FF01990C39052000F004FF0021072000F04EFFA6
:2052000006AE311D072000F049FF01990839052000F0F6FE0021072000F040FF3100083168
:20522000072000F03BFF0199091F052000F0E8FE0021072000F032FF0C363100072000F06D
:205240002DFF06988B4988420DD107988A49884209D108988949884205D1099888498842A4
:2052600001D16846057387492000FFF729FC1F21072000F0C5FE844F39002000FFF7F0FB04
:205280000021042000F00AFF6946072000F006FF02A9072000F002FF00200099890303D426
:2052A0000299090300D50120260079366946097B002956D0002800D099E0B078002827D141
:2052C00072492000FFF7CCFB0021042000F0E6FE05A9042000F0E2FEFF2505992943042029
:2052E00000F08EFE0021042000F0D8FE01A9042000F0D4FE01980540280001F0CEF8019049
:2053000008200199401AB0700599042000F078FE39002000FFF7A4FB02985D49014080201A
:205320004002084302900146072000F069FE009880B2009000200490564C00980107C90F61
:2053400007D008218843009001462143042000F057FE009807218843009004432100042037
:205360004DE0012500284DD0B94F0098384005430095484C29462143042000F041FE04984A
:2053800000282DD0009802210143009100992143042000F035FEAF48056A6D1D00210420DF
:2053A00000F07CFE6946042000F078FE0198800303D4A848006A281AF4D5009807400820EB
:2053C0003843009001462143042000F019FE009802218843009004432100042000F010FE4C
:2053E0000298B54901400291072000F009FE029C0121062000F004FEB0492140072000F0DA
:20540000FFFD18E00498C000B9490143019104980099C9080D40A84203D00199042000F0A6
:20542000EFFD01980221884301900146042000F0E7FD00F0C7FDAF480068002801D0FFF727
:20544000DFFA00F0BFFD0021032000F027FE6946097B7170C90701D50121F170002801D434
:20546000049931700BB0F0BDFF00010E50EF00E008ED00E04A4C494E4B4D4F4E48414E4407
:205480004C45520030ED00E0F0ED00E020ED00E0FFFFF3FF00005FA0F0B587B00400206D26
:2054A0009549884218D1200000F0D6FE002802D50020C043C9E0200000F0C8FEB4492000B9
:2054C000FFF7FEFA002807D40021072000F098FD002801D100F076FD26007A36AD4D307839
:2054E000002800D184E0AC492000FFF7B9FA0021042000F0D3FD04A9042000F0CFFD049863
:20550000C0B2049029002000FFF7AAFA002807D40021072000F0C2FD6946072000F0BEFD27
:2055200000988021C902014300910099072000F067FD684614210173012305AA03A9200088
:20554000FFF7DEFBAF4F0598384001900146049A0120082375785B1B9840101800020843F7
:205560000190012301AA03A92000FFF755FC009D0121062000F044FD50492940072000F089
:205580003FFD0021072000F089FD324D2E6AC83602A9072000F082FD002802D50020C04399
:2055A00008E002990803C00F02D1296A711AEFD502990091050041D40098A349014000913D
:2055C000072000F01DFD012301AA03A92000FFF797FB019807400598FF2109020140394312
:2055E0000191012301AA03A92000FFF715FC25E029002000FFF764FA9449072000F000FDE4
:205600009349072000F0FCFC00F09CFD114D2C6AA41C02A9072000F041FD002802D5002043
:20562000C04306E002998803C00F02D1296A611AEFD505002E49072000F0E2FC00F0C2FCC8
:205640000021032000F02AFD280007B0F0BD0000FFFF0000B801002002B582B069460F22C3
:205660000A70012302AAFFF723FC03B000BD70B582B00400774DC04E00290ED000F0B0FC8B
:20568000002060653068A84214D26946012000F005FD0099012081430AE03068A84209D236
:2056A0006946012000F0FAFC009801210143012000F0A6FC73BD0000FFFFFAFFFFFFF7FF68
:2056C00001290AD9091F0CD0091F04D008390AD0703904D009E0A9487047A94870471F20AD
:2056E0007047032070470120704700207047000003005FA03C120020FF00010EF0B583B014
:2057000005000F002C00503420689E4988423CD1002001909C492800FFF7D2F9002807D4FD
:205720000021072000F06CFC002801D100F04AFC964E0023320021002800FFF769F900209F
:20574000009001AB01223100200000F0BFFB0198C004840D641C01980001450C6D1C0126E6
:205760000320019A0240921C012191403E603871880000F0FBFEF871280000F0F7FE787171
:20578000200000F0F3FEB8713E74002003B0F0BD50EF00E0F0ED00E020ED00E0F0B583B00C
:2057A00005002C00503420687649884201D0002026E0B04E0023320021002800FFF728F979
:2057C0000020009001AB01223100200000F07EFB012701984008384012D0C14E00233200C9
:2057E00021002800FFF714F90020009001AB01223100200000F06AFB0198000C0740380014
:2058000003B0F0BDFF00FFFF38B5046D5D4DAC4217D1049CA4000919CC79A240202489797A
:20582000611A8B4013431C00AE49FFF749F9002807D42100072000F0E3FB002801D100F07E
:20584000C1FB002032BD0000FFFFFBFF0F005FA00D005FA0A6AE0000F5B585B00E00842A7C
:2058600002D20020C04385E0300050300190059840690290059880690490842200213000A2
:2058800000F034FE059800680090002801D1964800900098000E954CFF2808D0032801D067
:2058A0000E2804D100983749884200D0904C0598007B694608730598407B01061BD500219D
:2058C000820701D580218903420703D50A008021C9031143020703D50A0080210904114363
:2058E000800603D40800802149030143301D01677820012131540598807B002804D0202842
:2059000002D201248440641E351D0498042809D3029800F0CEFDE8660298001DA866E96E93
:2059200001F02EF937002C378020400000F01EFE2021785420370520787036606D48686045
:205940006D4828600020E86028616C49A96001996A46127B0A75019901228A7501998C60C3
:205960000199009A0A600199486078360598B0600698843807B0F0BD38120020370000800D
:2059800001000080FF00010E84ED00E080ED00E030B5C5B005000221684601F04DF96846C5
:2059A000018835A801F048F968460088042804D335A800F07EFD040000E04B4C9022002180
:2059C00001A800F093FD019401A80121017100214171017325A805904AA00890402225A971
:2059E00001A8FFF739FF01210598FFF740FE642D12D0652D14D06E2D16D06F2D18D0792D49
:205A00001AD07A2D1CD07B2D1ED07C2D20D0822D22D0832D24D026E001A801F027FA22E0D2
:205A200001A801F09BF91EE001A801F0DDFA1AE001A801F005FB16E001A801F027FB12E091
:205A400001A801F03AFB0EE001A801F03FFB0AE001A801F04BFB06E001A801F050FB02E03E
:205A600001A801F087FB00210598FFF700FE45B030BD000078ED00E070B582B00669012446
:205A800001207C21715C002929D01D493000FFF717F805000021072000F000FB0100294319
:205AA0000D006946052000F0F9FA284316D40098C00C204003D07C36002030700EE000983E
:205AC000000C04400AD10098802149020143072000F096FA6946052000F0E0FA002076BD3B
:205AE00014ED00E074EF00E0FF000003FF030000FF0F00009D570008FD56000809580008B0
:205B0000FCED00E0000000001D690008436A0008934D0008B14E0008295100089954000813
:205B20001D500008414F0008000000005956000859580008474B0008AF4B0008000000004C
:205B4000C15600080000000000000000000000006F560008795A0008F4B584B005000E008E
:205B60001F0000200290B80701D101200290287E421E9241D20F0221280000F0E7F9040037
:205B8000287D0106022000F03BFA00903100052000F036FA009908436968A14206D06C60D2
:205BA00005002100042000F02BFA2843002856D100F0C8FA002852D10498022847D3441E8D
:205BC0000A9E0298002826D0002E07D0F068B168401A844200D82000009000E000940025AE
:205BE0003900072000F05AFA002836D13F1D6D1C00988542F4D3002E09D0B06800994018B7
:205C0000B060F168884202D33000316888470098241AD9D11BE001A9072000F03FFA002847
:205C20001BD101983870010A7970010CB970000EF8703F1D002E08D0B068001DB060F16897
:205C4000884202D3300031688847641EE3D101A9032000F023FA002804D000F0C7F9002031
:205C6000C04304E00199380000F00EFC049805B0F0BDF5B583B00E001C00007E421E9241BB
:205C8000D20F0A9F3900039800F060F905000398007D0106022000F0B3F900903100052095
:205CA00000F0AEF90099084303994968A94208D003994D6000902900042000F0A1F9009910
:205CC0000843002835D100F03DFA002831D10498022828D3451E0120B84002906846032159
:205CE000C91B017001A9072000F0D8F9002802D000F07CF91DE001986A4612783240D1004B
:205D0000C840019001982070641C002F03D00198000A2070641C0398007E002801D10298DF
:205D200036186D1EDED101A9032000F0B7F9002802D00020C0430FE001980321C91B314050
:205D4000C900C840019001982070641C002F02D00198000A2070049805B0F0BDF3B583B02B
:205D600015001C000A9F012F01D1924804E0022F01D1914800E0012001900398007E421EA2
:205D80009241D20F7910039800F0E0F806000398007D0106022000F033F9009004990520AE
:205DA00000F02EF901000098014303984068B04209D00398466000913100042000F020F9B1
:205DC00001000098014300290CD1A00710D1042F0ED12168072000F013F9241D002804D558
:205DE00000F004F90020C04323E06D1EF1D119E02178022F0CDB0A00607801021143032F2E
:205E000006DB0A00A0780004E17809060143114301984143072000F0F3F80028E0D4E41983
:205E20006D1EE5D100F0CEF80021032000F036F9002005B0F0BDF9B581B00D001600807D87
:205E4000002802D10020C0433EE0002708980890099809900BE02000089988400199097ED8
:205E6000002900D12D18029908180290361B002E29D001988068A8430899C840401C019913
:205E8000097E002901D0340003E03400864200D904000898022808DB09980090029B2200F4
:205EA00029000198FFF758FE06E00090029B220029000198FFF7DDFE002801D5070002E025
:205EC0003F18A042C7D0380003B0F0BD10B582B0049C0094FFF740FE16BDF9B583B00D003A
:205EE000160000270A980A9001200A99884001900CE03F190A99200088400399097E0029F1
:205F000000D12D18049908180490361B002E1AD003988068A8430A99C840401C0399097E19
:205F2000002901D0340003E03400864200D9040001980090049B220029000398FFF70EFFC6
:205F40000028D6D50700380005B0F0BD78B403681A4CA34201D1012300E0002380256D04DC
:205F6000C468E60201D48225ED05260203D52E0080252D053543660203D52E008025ED041E
:205F80003543A60203D52E008025AD043543240305D5007C002802D12800094D0540002BA7
:205FA00003D128008025AD05054329431001084372BC70470101010101000100FF00010E85
:205FC000FFFFFFF380B56846FF21417000210170082300AA921C6946401C01F004FC01BD4E
:205FE00000B583B030236A4672A104E000B583B030236A4671A14F4801F0F5FB03B000BDDA
:020000040800F2
:20600000F0B58FB0002200240B0C4B401D0A5D402B096B409D085D4003916B086B40D9073D
:20602000C90F03AB1971444F3D6A6435434E6946305C08704A7009E084235B0005AA00BF26
:2060400060A100BF68A001F0CEFB641C0D2301AA69463000083001F0C6FB01A840784007F2
:20606000400F012808D1212301AA03A91036300001F0B9FB00200FE0022808D0042802D109
:20608000FFF7AEFF01E0022CD6DB002003E0386A281ADBD50120C0430FB0F0BDF2B58EB091
:2060A0000021002502AA1171254F01AA385C107051702148066A643608E084235B0004AA6D
:2060C00040A100BF48A001F08EFB6D1C0D236A4601A93800083001F086FB68464078440718
:2060E000640F012C13D1C006840F21236A4602A90A37380001F077FB0E98002804D000980E
:20610000800004430E98046000200FB0F0BD022C09D0042C02D1FFF763FF01E0022DCCDB09
:206120000020C043F1E70448006A301ACED50120F7E70000F8020020B8010020E0020020CD
:20614000D002002080B500210720FFF7A7FF02BD00B58BB084235B0001AA00BF19A100BFA0
:2061600021A001F040FB69460020FFF797FF002811D469460120FFF791FF0098B2210140C8
:206180000BD0FFF72DFF69460120FFF787FF0098A021014001D0012009E0A021C905009121
:2061A0000120FFF72DFF401E8041C043C00F0BB000BD000081C003000000000081E003008B
:2061C00000200000FFFFFFFFFFFFFF9EE7FFFFFFFFFFFFFFB6EDFFFFFFFFFFFFFF0000A5E7
:2061E0000000000000000000FFFFFFFFFFFFFFFFFFFFFFFFFFFFFFFFFFFFFFFFFFFFFFFFB7
:20620000FFFFFFFF00000000F0000000F8B403008818401E1F22D24311400240501A420947
:20622000521C49090124C9B2C8081D182C20285C01264F077F0FBE4006432C352E70491C73
:20624000521EF0D14E331C70F1BC704700B520212C3001F085FB00BDF1B588B04E30007848
:20626000002800D1B8E008984E300021017008988168080000D1AFE00898006888470028ED
:2062800000D1A9E008984268100007D008991831089800689047002800D59AE00898016929
:2062A000080005D0089800688847002800D590E00020039008980190012405E00398401CD8
:2062C00003900198001D0190039808998969884276DA0198007F022803D0032801D004285F
:2062E000ECD10198C07F08994D310978401A0490002008994C310978019A527F8A4200D2B2
:20630000881A00210291049901228A40069201218140059118E00898C66830000AD0039821
:2063200000902B00029A0899183108980068B04700284ED46D1C0198817F01208840854201
:20634000E9DB0298401C029002990198427F012090408142B2DA08460499884008994C31EB
:206360000A7801219140491E0140002205980128E7DB03460800069D012D0CDBC608089FD8
:20638000BE192C36367847077F0F3E41264002D1401C6D1EF2D1921910D10198407F049D53
:2063A00045190120A840081808994C310D780121A940491E01405B1EC3D0DBE70025BAE76C
:2063C00008984169080007D0089800688847002802D50020C04300E0002009B0F0BD38B449
:2063E000012100220368001D002B0BD00468001D0C4202D04D466D1E64192260241D1B1F8A
:20640000F0D0FAE732BC704701680A060B0A1B061B0A13430A02120E12021A43090E114304
:20642000016070470106020A1206120A0A430102090E09021143000E08437047CA088218BB
:206440004807400F9107C90E4118032082431068002906D0C840030050682022511A88403F
:206460001843704702681170090A5170921C0260704702681170090A5170090A9170090A9E
:20648000D170121D026070470170090A4170090A8170C01C090A01707047010006D000202C
:2064A00001E04908401CCA07FBD570470020C04370470178427812020A438178090411432E
:2064C000C07800060843704718B4012A0BDB0300401C0C00491C1B782478A34201D00120C9
:2064E00002E0521EF3D1002012BC7047012A03DB0170401C521EFBD1704778B403000020C9
:20650000002480252D0601E03100641C294202D14E00B342F8D2002C09D440008B4203D3B6
:206520005B1A0500012028434908641EF5D5002A00D0136072BC704780B56A46FFF7DDFFAF
:20654000009802BD80B50022FFF7D7FF02BD80B5002807D5002243421800FFF7CEFF010046
:20656000484202BD0022FFF7C8FF02BD002101E0491C4000002800D4FAD11F20401A704776
:206580000278401C0B78491C002A01D09A42F7D0D01A704738B472B6A54A90680021117160
:2065A00062B6002823D00168002920D043694C699C421CD100E021000C68002C02D06569B9
:2065C0009D42F8D072B603681469844200D11361026A13601A6201620A680260002A00D06D
:2065E0001062086038200A00393212780A5462B631BC7047F8B500278D4C6770012020701B
:2066000072B6E06B010004D08047E76367633820275462B601F0A6F90078CD2802D07D2000
:2066200001F0A6F9A068002807D0C16B002904D009680A0001D0406888473120205C0028E2
:2066400009D0A06838303021615C01702079002801D0FFF79FFFA068002805D0017C0029A1
:2066600002D1416B491C41632069002826D002E02868206162B672B62569002D41D02E7C42
:20668000002E3ED070070FD5E868216A411A012906DA280000F090F8287C002804D10DE0F5
:2066A000616A411A00D56062FB2030401028DFD1A86880684068007C0028D9D172B620E094
:2066C0002069002804D0686921694969884218D3287C400710D5E868216A401A012806DA65
:2066E000280000F069F872B6287C002809D0E868616A411A00D5606262B62D68002D72B645
:20670000DED1607900280BD12069002832D02069007C0028206911D08068806840680DE03E
:206720006771206A8021C90540186062E169080001D02000884762B6E568DFE7A060C06A07
:206740000078CD2802D0782001F012F9A068C16B002904D049680A0001D040688847A0682A
:206760003030017A3022A1543122A1540168491C016006E03120275430202754A760277065
:2067800062B62000F2BD10B5294C2078401E2070207800280FD1606800280CD072B606D0E8
:2067A00001202070200001F051F9002020706078002800D162B610BD38B581681C4C002900
:2067C00009D0226AC2600A684968002A00D051600A6000218160017C8907890F017413D1FA
:2067E0002169002911D1206101202178002906D12070200001F02AF90020207000E06071A4
:206800006078002800D162B631BD42694B699342E9D38142E8D09A42F6D103001B68002BE2
:20682000EED05D69AA42EBD18B42F7D1DBE70000B801002038B54169304C2278521C22704F
:2068400022000C3200E01A001368002B02D05D69A942F8D3036002621060002B09D0186235
:206860005A698A4202D13921415C00E0002138228154017C002906D172B6FFF79DFF607880
:20688000002800D162B6FFF77EFF31BD38B51B4C25782078401C2070200001F0D7F825709C
:2068A0006078002800D162B631BD10B501F0FCF812480121017001F055F8040001F056F8E9
:2068C000021B203A012A03DBCD212000FFF70EFE10BD80B509490A6A80180A78002A04D048
:2068E00062B60A6A121A07D5FBE772B68968C86004200874FFF7CAFF01BD0000B8010020EB
:20690000402801D32B3806E0212801D1142002E0142800D11320C0B27047FEE7FDB584B08D
:206920000D0014469549194002910C9E0D980D90E80715D5002C13D00D98019002980090F2
:2069400033000122290004980069049FFF693F6BB847002873D4241A01286ED1761C6D1CCF
:206960000698400057D4A80718D5022C16D30D980190029801210143009133000122290015
:2069800004980069049FFF693F6BB847002856D44100641A012850D1B61CAD1C0698002882
:2069A0001CD4042C1AD3A00803900D98019002980221014300913300039A290004980069C9
:2069C000049FFF693F6BB847002838D48100641A0399884231D1880036182D18022C1AD332
:2069E000600803900D98019002980121014300913300039A290004980069049FFF693F6B22
:206A0000B84700281BD44100641A0399884214D1480036182D18002C0FD00D9801900298A0
:206A2000009033002200290004980069049DED692D6BA847002802D4241A0598001B07B01A
:206A4000F0BDFDB584B00D0014464C49194001910C9EE80713D5002C11D000913300012247
:206A6000290004980069049FFF697F6BB847002800D581E0241A01287CD1761C6D1C069829
:206A8000400067D4A80716D5022C14D3019801210143009133000122290004980069049F15
:206AA000FF697F6BB847002866D44100641A012860D1B61CAD1C0698002830D4042C2ED374
:206AC0000498C069876B38000FD0019800280CD100903300A208290004980069B847002888
:206AE0004AD48000241A2D183618A008029016D001980221014300913300029A29000498E2
:206B00000069049FFF697F6BB847002834D48100641A029988422DD1880036182D18022C3D
:206B200018D36008029001980121014300913300029A290004980069049FFF697F6BB847EF
:206B4000002819D44100641A0299884212D1480036182D18002C0DD00198009033002200B7
:206B6000290004980069049DED696D6BA847002802D4241A0598001B07B0F0BD0000FF3F93
:206B80007047FEE7002804D00021002206C00838016070476E48012101707047002900D102
:206BA000704780B5002803D06A4A12685269904701BD70B588B004002022C9B26846FFF7AE
:206BC00095FC644D212C01D3202600E02600310068462A6852699047A41BF3D108B070BD9B
:206BE00080B50021FFF7E5FF01BD80B5594A12689269904701BD01B501216846FFF7CEFF7C
:206C000001BD01B502216846FFF7C8FF01BD01B504216846FFF7C2FF01BD68464D4A1268F7
:206C2000D269904701BD01B50421F6E780B549480068006A804701BD80B5002901D100205F
:206C400002BD444A12689268904702BD50B589B00400212C01D3202600E02600310068464F
:206C6000FFF7EAFF002801D1A41BF2D109B050BD80B5384A1268D268904702BD80B5042198
:206C8000FFF7DAFF02BD10B582B00400684600220260FFF7D1FF69460A784B781B0213430C
:206CA0008A7812041A43C97809061143216016BD80B5284800680068804702BD80B52548CA
:206CC00000684068804702BD10B5224C201D00F0F9FE00F085FF2048206010BD80B51D4804
:206CE000001D01F0CBF801BD80B5194800210170184800680069804701BD80B501F0A7F862
:206D000002BD10B582B0040004E002211148001D01F0DAF801F09BF800280BD001F092F877
:206D2000012807DB0B480C49016001212000FFF783FF16BD01F08BF80028E6D00021684691
:206D400001F068F80028E0D50020C04316BD00005D1B0020300B002040F90008F1B58AB0FB
:206D60000024E443082108A8FFF766FF089806900998010C0904079180B20590019001F0C2
:206D8000EEF80599814200D90100029108469349884202D3FF2188430290029801F0EEF888
:206DA0000490002803D13EE00698001906900198002801D1059C3EE006460298864200D9FF
:206DC00006000198801B0190069F002531000498FFF74EFF0395FFF76BFF311A039A8C1A88
:206DE000002803D0402CF6D33F208443002D0ED1049988180090079B220039000A98C56997
:206E0000AD68A8470500A54200D100253F19039800190390B042DED1002D02D00024E44302
:206E200001E03400C0D50198002801D0FFF70EFF0498002802D0049801F0C6F82000FFF71C
:206E4000E6FE0BB0F0BD38B50500AC683F2084430BD0210028696A681018FFF7C6FE2869E8
:206E600000192861A868001BA86031BDF1B592B0082106A8FFF7E0FE069F0798010C09045E
:206E8000059180B20490044611280ED301F067F803900498001D0399884200D20390039830
:206EA00001F06CF80290002803D10DA8029014200390039E361FA64205D24948864203D3FD
:206EC000760A760200E0260046480890802080000B900298099000200A900C9008A8019009
:206EE00002980090059B320039001298C5696D68A84705000C98012D02DA241A1FD121E0DF
:206F00007F19641B291A0091002C0ED1049902984019FFF7B9FA0099091D0C98029A10181B
:206F2000FFF763FEFFF782FE0FE0029A1018FFF75CFEFFF77BFEB542BBD00498051B2000B4
:206F4000FFF74EFE2800FFF762FE02980DA9884201D001F039F813B0F0BDF0B5D3B00400C8
:206F600005216846FFF768FE6D46297802A8FFF763FE687800281ED0A87800280DD0A54E7E
:206F8000316A0F182069E169096A8847002808D1306A381AF6D5002003E02069E169096A19
:206FA00088471290012808DA1298012810DB28788100091D0DE0012012902B7812AA121D12
:206FC00002A92069E469E468A0470028ECD51290042112A8FFF7E2FD53B0F0BD01100000FD
:206FE00001040000476E000870B5D4B0060002E001A8FFF7D3FD002442AD01216846FFF7F6
:207000001BFE68460078FF2806D0684600782870641C6D1C402CF0D1230001AA42A93069EE
:20702000F569ED68A847A1006A461278FF2ADFD101AA5050091D01A8FFF7B0FD54B070BD0C
:20704000F0B5D3B00700002442AE02AD0BE0042101A8FFF7F1FD68460078307001982860BA
:20706000641C2D1D761C01216846FFF7E5FD68460078FF28EBD1230002AA42A93869FC6943
:207080002469A047FFF7C3FD53B0F0BD10B582B0040001216846FFF7CFFD684601782069D9
:2070A000E26952699047FFF7B2FDE06D002803D00121200001F02BF913BD80B50100086938
:2070C000C96989698847FFF7A2FD01BD10B504002069E169C9698847FFF799FDE06D0028CC
:2070E00003D00021200001F012F910BD80B501000869C969096A8847FFF789FD01BD10B599
:2071000084B004000020039014210291019004E06846017803A8FFF78FFD01216846FFF72D
:207120008BFD6846007800280AD1039B019A02992069E469646AA047FFF769FD04B010BD62
:20714000012100A8401CFFF777FD684640780128DED00AD3032804D007D26846017802A8DC
:20716000D9E76846017801A8D5E768460078FFF76DFDD2E710B584B00400002003900120B3
:207180000290019004E06846017803A8FFF754FD01216846FFF750FD6846007800281FD17E
:2071A00003992069E269926A90471A480178491C01700120FFF78DFB01992069E269526913
:2071C00090470298FFF785FB2069E169C96988470400FFF7D8FA2000FFF719FD04B010BD7B
:2071E000012100A8401CFFF727FD684640780428C9D00AD3062804D007D26846017802A89B
:20720000C4E76846017801A8C0E768460078FFF71DFDBDE7B8010020FDB586B00291069D7B
:207220001035296904916846848B0E980E90AE8A0641AF48006A6A46128C80180390002E5A
:207240001FD02700B44200D937000E983A0082400092029801F052F9F61B0E98310081405F
:207260000191002E06D00A46009804990918286901F044F90198A88200980299081802906B
:20728000E41B002C1BD00E9801906846008C00906846838B029A00212868EE68B66CB0475F
:2072A000002800D50020241A0E99884002990818029003988E49096A401A0128E1DA0E98EE
:2072C000E88206988C30012101706846808B001B09B0F0BD30B583B00500042101A8FFF73C
:2072E000ABFC00F03CFE0199814202D300F037FE01900198052815D300F040FE04000020D5
:20730000009000230198021F92B2211D2800FFF783FF2060011D2000FFF740FC200000F0DE
:2073200053FE02E00020FFF772FC03B030BDF0B585B00700082103A8FFF77EFC03AC20887A
:207340008000E188884200DA0800001D00F016FE0500E18809D10800FFF778FC654802907E
:20736000042102A8FFF71AFC33E0002901D0FFF763FC0026607900280AD102200090638831
:207380002288291D3800FFF747FF0290064614E0012810D10220388523880190608800901A
:2073A000E0888010C01A80002A1801213869FC69A46CA04700E0C048029002992800FFF7E7
:2073C00063F8B100091D2800FFF7E8FB280000F0FBFD05B0F0BD10B582B00400012168463D
:2073E000FFF72AFC684601782069E269D26B9047FFF70DFC13BD1CB5040008216846FFF7F1
:207400001BFC00200099012905D1019901220A438834226000E0A848FFF7F9FB13BD10B505
:2074200003000120002900D0C148002B5CD05968002902D00100022008439968002902D0A9
:20744000010004200843D9680C0002D00400082020431C69002C02D00400102020435C692F
:20746000002C02D00400202020439C69002C02D0040040202043DC69002C02D004008020B6
:2074800020431C6A002C03D004008020400020435C6A002C03D004008020800020439C6A6B
:2074A000002C03D004008020C0002043DC6B002C03D00400802040012043002903D001007B
:2074C000802080010843996C002903D001009020C00108430100C020400208435B6C190034
:2074E00002D0010010009847FFF791FB10BD0000B8010020F9FEFFFF00B583B0012100A8FB
:20750000401CFFF799FB01216846FFF795FB0220FFF79CFB00280CD101A968464078000269
:207520006A461278104301F017F800220199FFF776FF03B000BD00B583B0012100A8401C19
:20754000FFF77AFB01216846FFF776FB042102A8FFF772FB01A96846407800026A4612780B
:20756000104300F0F9FF029A0199FFF758FF03B000BD70B5A6B09022002101A8FEF7B6FF3C
:20758000012100A8801CFFF757FB01AD04E06846017801A8FFF777FB01216846FFF74CFB66
:2075A00068460078002806D101A96846807801F05AF826B070BD012100A8401CFFF73CFBBD
:2075C000684640780728E2D031D3092809D002D30A280AD02BE068460178281DFFF72CFBE1
:2075E000DAE768460178681DF8E768460078082802D26846047800E008242100280008305E
:20760000FFF71AFB68460078061BC5D0300000F0B5FC0690002804D03100FFF70DFB079654
:20762000BAE768460078001BFFF710FBB4E768460078F9E770B582B002216846FFF7FCFAB2
:20764000684646780078C100091809014F4A541804282DDA25001035E968002928D0112E07
:2076600026D2C100081A8000494908184949096AC1602868002802D1200000F084FF8C200D
:2076800001212154E868C26CB00000BF43A10E5810000AD00121286890472000B047002171
:2076A0002868EA68D26C904773BD2000B04773BDFFF770FA73BD0000FAFEFFFFF8B5012008
:2076C0000090324F3C00324D0C358D3704262069002825D08C20205C002821D038780028F0
:2076E0001ED128682C4940182A49096A401A012816DB200000F03EFE002800D100902000EF
:2077000001F074F9002800D1009020001030C068016D080004D020008847002800D1009038
:20772000903490371C35761ED1D10098F2BD0000010000400100401C0022D243914201D176
:2077400000210420CA0052181201104B9A181369002B02D08C3200231370491C8142F1DBBF
:20776000704738B50C0000280FD4C1000818000106490D18002C03D1280000F0A4FD02E05D
:20778000280000F0B4FD8D352C7031BDC812002048120020B8010020102700006D6E00086D
:2077A0005D6D0008E96F0008417000088D700008BB700008CD700008ED700008FF70000885
:2077C00075710008D5720008D77300085B6F00082F73000881840008E18D0008F7730008A9
:2077E000F0B5059C02E0F0B5334C2468A6464C4655465E466746F0B4994682468B46944651
:207800002E4A10210420148801263602B4432304344323437446012C00DA51E04F46092FE6
:2078200000D308275C4625782D02641CA34654462678641CA24635436C0810D31A266C0A4A
:2078400000D318269153138010836D08744600BF641EFDD550837446641EFDD510E01C0CD2
:20786000148010836D087446641EFDD550837446641EFDD51469640902D30124E405254348
:207880007F1ED9D14E46082E02D20824A41BE5402D0C64462570641CA4464E46092E02DB69
:2078A000083EB146BAD1F0BCA146AA46B346BC461C0C1480F0BD0000EC0A002000000048BB
:2078C0004F46092F00D308275C4625782D02641CA34654462678641CA24635436C0809D39A
:2078E0001A266C0A00D318269153138010836D0850830AE01C0C148010836D085083146971
:20790000640902D30124E40525437F1EE6D14E46082E02D20824A41BE5402D0C6446257035
:20792000641CA4464E46092EBDDB083EB146C7D1130030B414001500103902D310393CC022
:20794000FCD2490700D30CC000D504C0890002D30280801C002900D5027030BC7047000042
:207960000022E5E700487047601B00206846704706490A78521C0A7000224A7062B6044920
:20798000087008780028FCD1704700BFB8010020551B002038488168002901D108B00ED021
:2079A000EFF30982283A0368F8C243464C4655465E4678C2734608C2283A83685A60FEF7C0
:2079C00019FE816800291CD04A68143278CAB346AA46A146984608CA9E46283AF8CA274960
:2079E0000B60143282F30988704604210843864690692349814203D02248034200D162B64B
:207A00007047214821490968401A80F308882049C161204981610621C9438E46704701BCBD
:207A200020461D498E4600BDFEE71C48006817490968401A20380721884380F3088800219E
:207A40000D48417062B600F012F8FEE703680CB40021417062B61249124A0A6000BF72B60C
:207A60000CBC036070470E490E4A0A6070470C490C4A0A6070470000B8010020B8010020D6
:207A80005E7A000800FF0000401D00203CFA000800000001D1F70008297A00080048000880
:207AA00004ED00E000000010EFF3108072B604490A68FF231B0413430B6080F310887047C8
:207AC00020ED00E010B572B6074C6178491C617008220021FEF70AFD6078401E6070607845
:207AE000002800D162B610BDB801002080B5B84801210170002001F063FB01F031FB01BDBD
:207B0000F0B583B0002069460880142401F07CFB002800D0102401F075FB002801D01820D8
:207B200084430122012100A8801C01F0AFFB68468078012802D0022806D00BE00422002187
:207B400001A801F039FC15E00422082101A801F09DFB0FE0AE480190102C0BD1012200210E
:207B6000684601F093FB68460078042802D26846012141700198BB4F3E000B360C2502AA32
:207B80000A21FEF7BAFC029930313170761E6D1EF5D1FF20801C69464978002903D06946B7
:207BA000097808180CE0102C0AD0142C01D1001D06E0042C01D1401D02E080204001204388
:207BC000788203B0F0BD80B5FFF788F801BD8807800F022800D1704780B5FFF77FF801BDB2
:207BE00030B583B0FFF78CFF01F098FD02F0E8FB9C4C01F007FB00281FD101AD009000233D
:207C000040220221012001F0EEFC28704020009023002C3340220221002001F0E4FC68708B
:207C200001A802F085FC9049002002F0B8FC00228E492000203002F0E3F81034200002F0FD
:207C4000BCFA01F09EFD03B030BD80B501F0BFFA1420FEF73EFE01F0B9FA01BDF2B582B0C3
:207C600083490978002948D10600029C80484568002D20D04020401B2700844200D90700B7
:207C80003A0031007A4840190C3000F037FCED19F619E41B402D0ED17648006800900023C6
:207CA000402273490C31002002F0F2FB402801D0FFF71CFF0025A709BF010ED06D48006890
:207CC000009000233A003100002002F0E1FBB84201D0FFF70BFFF619E41B002C06D022009B
:207CE000310063480C3000F009FC2500604845608068029940185E49886003B0F0BD38B54E
:207D0000334C207800281BD162685A4D2B68002A0BD021000C3102F0B1FB6168884201D0CF
:207D2000FFF7E4FE0020606008E000930123002102F0AEFB2968002002F039FC0020A06038
:207D400031BD38B505000C002148007800280CD1FFF7D5FF4748036822002900002002F030
:207D60008DFBA04201D0FFF7C1FE31BDF8B507000D00174C2078002828D162683D4E002AC9
:207D80000BD0336821000C3102F078FB6168884201D0FFF7ABFE00206060316802F00EFC32
:207DA000002801D0FFF7A2FE0023DB432A003900002002F063FB002801D5FFF797FEA806E9
:207DC00001D0002001E0A0684019A060F1BD00003C0B002038B505000C0025480078002850
:207DE00007D0220000212800FEF780FB0020C04332BD2048036822002900002002F071FB23
:207E0000A04202D0FFF772FEEBE7002032BD000040E2010080B5164A1278002A02D0002009
:207E2000C04302BD0A000100002002F062FB02BD80B5002002F074FB02BD80B5002002F08B
:207E400068FB02BD80B5002002F05BFB02BD80B502F016F88007800F022801D1012002BD7D
:207E6000002002BD48010020C77B0008CF7B00083C0B0020440100204020704738B504004A
:207E800072B6104D6878401C687001202071206800280ED02878401C2870200002F0A6FBC2
:207EA000002804D16079012801D000202071FEF76AFC6878401E68706878002800D162B6DF
:207EC00031BD00BFB801002070B5040072B60F4E306A4518207900280CD12A004821200026
:207EE00002F0A8FBB068C068281A012801DA012070BD72B66079012801D000202071707885
:207F0000002800D162B6002070BD00BFB801002018B40022426001602A490A68002A02D198
:207F2000086011BC70470A0000E0221D1468002C01D0A042F9D24460106008680028F0D09A
:207F400000E0080041680029EBD0026883188B42F7D14B684360096851180160F2E7002088
:207F60001849096804E00A68904200D2100049680029F8D1002800D00838704718B40100C6
:207F80000020C91D0722914308310E4A00E01A1D1368002B14D01C68A14208D218005B18E0
:207FA00013600268521A1A6042685A6004E08C42EDD118005B681360002801D0016008304A
:207FC00012BC70472C0B0020002800D1704780B508380168FFF79CFF01BD80B5CA1D0721A4
:207FE0008A430832083801680260891A8018FFF78FFF01BD10B504002068FFF7E5FF0020A7
:020000040800F2
:20800000206010BD80B507229143FFF781FF01BDF2B504001500666E216E891B012901DAE1
:20802000626D89188D4228DA616DE26D5118881B2F00854200DD0700002F1DD03A0000990D
:20804000300000F05BFAF6190098C0190090ED1BE06D616D41188E4200D10600002D0BD070
:208060002A000099300000F049FA7619E06D616D41188E4200D106006666F1BD7CB5040081
:20808000042101A8FFF7A6FEE06D002802D1FEF7BEFD73BD256C0198290002F005FB684360
:2080A0000190206E616E814201D3081A02E0626D101A40180199884200D9080000900421EC
:2080C0006846FEF76BFD0098002826D0256E02F019FB606DE16D0818461B0098B04200D24E
:2080E0000646002E07D031002800FEF757FDAD190098801B0090E06D616D41188D4200D1F0
:2081000005000098002805D001462800FEF746FD00982D1802F0FBFA256673BDF0B585B0C5
:2081200004000026039604213430FFF753FEE662606B0B2805D20001FFF720FFE06200280F
:2081400022D10120C0430390606B00010830FEF77DFDE06A002802D0FFF736FFE662E06DFE
:20816000002801D0FFF730FF206B002801D0FFF72BFF3C2200212C342000FEF7B7F90398FE
:20818000FEF745FD05B0F0BD616B0901FFF722FE042120003830FFF71DFE042120003C30EB
:2081A000FFF718FE276C2664606B012808DBE16A091D226C0B68D21822641031401EF8D175
:2081C000206C001D2064AC494843A16B02F06CFA0500E06D002806D0616DA94216D0FFF7A9
:2081E000F3FE6665E665FFF7BAFE216C0091400802F05AFA00994843854200D9050028002D
:20820000FFF7BCFEE06500280FD06565206B002805D0216C8F420CD0FFF7D6FE2663206CF7
:20822000FFF7ACFE2063002803D10120C04303908FE7A665E06D2066E06D60663C20205C29
:20824000C0070AD502F092FA0500A06B2F182800FA21890002F014FA08E08848056AA06BA5
:20826000FA21890002F020FA2F1828002065A56467640496256B042204A9280000F03EF93A
:208280002D1D0295002515E02801E16A0E180020019002980090B368726831682000E76970
:2082A0007F68B8477168884200D068E70298401802906D1C606B8542E6DB226C216B20007C
:2082C000FFF7A6FE5BE710B504000120A16D01400CD1E16B084002D002F048FA01E0674882
:2082E000006AA16C0818E16C401AA06410BD10B504000120A16D014008D1E16B084002D0F7
:2083000002F034FA01E05D48006AE06410BD8D22825C002A00D0704738B53C300400227807
:20832000D007C00F00290FD10125E169294020D1002802D002F01AFA01E05048006A206160
:20834000E0690543E56131BD012912D1217FC9070FD5002802D002F009FA01E04748006A2E
:20836000E16808182169401AE060E06901218843E06131BDF0B585B0040001250495606BA3
:20838000002875D0206C002872D000270497E06B284003D002F0EAF9060001E03748066A87
:2083A000606C801B012863DAA16BE26B2A4007D100900800FA21890002F076F9010000981F
:2083C000401800D50020301860642C4E306A216D814218D020652069E169096A8847002835
:2083E00007D1A06D284012D001212000FFF78FFF0DE001283CD1A06D054039D100212000C8
:20840000FFF785FF34E0A06D2840C00730D4E06B054002D002F0AAF900E0306AA16C401AB6
:208420000390256B042203A9280000F067F82D1D0295002514E02801E16A0E18002001908B
:2084400002980090B368726831682000E7697F68B847716888420BD10298401802906D1C82
:20846000606B8542E7DB226C216B2000FFF7D0FD049805B0F0BD0000A0860100B8010020AD
:2084800010B58AB0040001216846FFF7A3FC6846007800281DD0022807D002D3032814D054
:2084A00027E02000FFF73AFE23E02000343000210160C16A026B8A4201D3501A02E0006A70
:2084C000401A8018FEF7A3FB13E02000FFF7D6FD0FE001900A210291FA2189000391049031
:2084E00005900690079008900990242101A8FEF755FB8C34012020700AB010BD124207D033
:208500008B0706D00B78491C0370401C521EF7D87047830706D00B78491C0370401C521EBF
:20852000F9D1704770B4103A03D378C9103A78C0FBD2530701D318C918C001D508C908C090
:20854000D20704D30B880380891C801C002A01D50B78037070BC704718B40200002300202A
:20856000FF24A41CA24208D0694CA24205D0694CA24202D0684CA24200D16848002900D071
:208580000B6012BC704770B50600FFF7E8FC050080204001854202DAFFF7E1FC0500002D58
:2085A00025D02800FFF7EAFC04002A0021003000F369DB6A9847002816D4291A2000FFF758
:2085C0000CFD34610020B0843062F069006800280DD0FFF7C4FC0100F0690068814206DB35
:2085E000FFF7CCFC306270BD2000FFF7EDFC70BD38B5C1000818000149490C18206900289C
:2086000030D0206A002803D020002030FFF7F2FCE06D0025002802D0FFF7D6FCE565E06AB9
:20862000002802D0FFF7D0FCE562206B002802D0FFF7CAFC2563606F002802D0FFF7C4FCEF
:208640006567A06E002802D0FFF7BEFCA5666069002803D020001430FFF7CCFC1034200041
:20866000FFF7C8FC31BDF8B50C00042826DA2168090E0025FF2900D100210E0221790E4393
:20868000C10009180901264A5718FFF7B1FFFF20801C864208D01E48864205D01D488642DE
:2086A00002D01D48864200D11C4DE561902221003800FFF737FF3800FFF765FFF1BD30B5DF
:2086C00083B00400164800250195009313000A002100C4696468A04703B030BD10B582B002
:2086E00004000F48009313000A002100C469A468A04716BD80B50A490869C969096A8847EE
:2087000002BD80B506490869C969C969884702BD0103000001060000010E0000045B000832
:20872000C8120020010088684A68801A01D5C96840187047010048688A68801A401E01D57B
:20874000C96840187047F2B504001500FFF7F2FFA84203DA2000FFF7EDFF05002E00A0682E
:20876000E16822685118091A37008E4200DD0F003A000099FFF7C2FEA068C0190099C919C2
:208780000091F61B2168E2688A18121A00D10800A060002EE3D12800F2BDF8B504000D0046
:2087A00001F0B0FF8F4F381D02F050F86068E168226851180E1AB54200DA2E00002E03D080
:2087C0003100FEF7EBF9AD1B002D03D029002068FEF7E4F9AD192000FFF7A4FFA84203DAFE
:2087E0002000FFF79FFF00E02800002810D00500E1682068411862688B1A9D4200DC2B0031
:20880000D2186260ED1A891A00D16060002DEFD1381D02F03BF801F07AFF2000FFF782FF09
:20882000050061682068E2688218521AAA4208DB012D02DB2A0002F041F8206860604019C2
:20884000A060F1BDF0B583B0050016001C00089B0020019000942800EF697F68B847B0421B
:2088600002D00020C0432AE06879002826D06069FDF7D8FD60612069FDF7D4FD206118348C
:20888000002618E02068FDF7CDFD20606068FDF7C9FD6060A068FDF7C5FDA060E068FDF7B8
:2088A000C1FDE0602069FDF7BDFD20616069FDF7B9FD6061761CE86E8642E3DB002003B08D
:2088C000F0BDF0B583B00400002708216846FEF7B3F90198012860DB0025434EA6422ED0D7
:2088E000B06E00282BD0706F002828D030682168884224D130792179884220D10422210013
:2089000008313000083001F0ECFF002817D1E8004019000134490D18686F002802D0FFF71F
:2089200053FB6F67A86E002802D0FFF74DFBAF662022002168352800FDF7D8FD03E06D1C53
:208940009036042DCADB656F002D0CD02800FFF73BFBA06EFFF738FB2022002120006830F8
:20896000FDF7C4FD0025019841000E18F6003000FFF704FBA06632000021FDF7B7FDA06EF3
:2089800000280CD0FFF7EBFA052101F08DFE0600FFF7F4FA050019D10127FF4306E0012705
:2089A000FF43002D07D02800FFF70EFBA06E002801D0FFF709FB2022002168342000FDF736
:2089C00095FD3800FEF723F903B0F0BD009820670198E066802026506567A567E56784346C
:2089E0002770EEE7080C0020C8120020F1B590B0614E3068002804D101203060301D01F0C4
:208A000010FF1098743002901098C06E002800D124E102980068002800D11FE1109884303E
:208A20000078002800D019E110980068000E082803D00C2801D00F2801D1022000E000207B
:208A400000060E900298FFF775FE042849DAFFF786FA05900298C0680599884200D3FDE03B
:208A60000846FFF78BFA040000D1B4E1301D01F0EDFE0298416882688A420AD3521A200038
:208A8000FFF73CFD0298806802994968401A201817E0C26803689A18551A2A002000FFF75A
:208AA0002DFD029801688068421A6019FFF726FD0298C06802998968029A5268891A6118F3
:208AC00008180299886002994C6002980599C16002980068FFF778FA02980460301D01F0AD
:208AE000D5FE1098C06E41000D18ED0018352800FFF744FA040000D199E00E98009023002A
:208B00002A001098016FFFF79DFE00280DD4207853280AD16078452807D1A078472804D112
:208B20001098C06E2169814203D02000FFF74CFA51E12100183103911099896E019100225F
:208B40000092012843DB002200258E68002E039B14D19B68002B34D0A04DAB4200DBD24352
:208B6000039D2D69AB4201DA0022D243039DED68AB4259DB1EE000BF080C00205B684F683F
:208B8000BB4200D0D243039B9B68B34201D00022D243039E3669B34201DA0022D243039E6D
:208BA000F668B34201DA0022D243039B1B680E68B34200D00125002A35D1002D01D001227D
:208BC00000921831039A18320392401EBBD1206941000A18D200210018310198FFF78EFC13
:208BE0002000FFF7F1F9009800282DD0206941000C18E4006846FF210174029806A96CC826
:208C00006CC106A8FFF796FD844204A811DA4470200A04A98870032206A8FFF794FD220094
:208C20001098816E0AE0CAD52000FFF7CDF90020CFE0002141708170032204A906A8FFF730
:208C400082FD0298089981601098806E039000270298FFF76FFD0400042C01DA0120B8E065
:208C6000039840680A900399096941180B91039AD26880180C90039880680D900398183006
:208C800003900D98002800D19CE00F919848844200DB441EE41E0AA8FFF744FDA04203DAFA
:208CA0000AA8FFF73FFD0400002C00D593E000D188E0029806A96CC86CC16846077404A8A0
:208CC0004470201204A98870032206A8FFF73BFD08980999069A5118091A25008C4200DDCA
:208CE0000D000B990D9A0A9B9A18521A954200DB15000022019200900E9B2A001098C669A3
:208D00007668B0470600AE4265D106A8FFF712FDA84203DA06A8FFF70DFD00E02800099980
:208D2000069A5118089BCA1A904200DC02009B180893801AC91A01D1069908910028EED137
:208D40000AA8FFF7EFFCA84203DA0AA8FFF7EAFC00E02800002810D00D990A9A51180B9BC2
:208D6000CA1A904200DC02009B180B93801AC91A01D10A990B910028EED1641BA8D1002E73
:208D800029D40298089981600B980F99884219D07900C919C900109A126F8C1828340A99CA
:208DA000401A059010984079002802D005A8FDF72BFB05A800900E9B042221001098C469A0
:208DC000A468A04700207F1C1099C96E8F4200DA3EE711B0F0BD0020C043FAE701000001C1
:208DE00070B584B0040043480168002904D101210160001D01F015FD012102A8FEF7EAFFD7
:208E00006846007A05286ED801A1095C8F4400BF06141C28728A0320009004216846FDF74A
:208E2000BDFE60E02000FFF74CFD5CE020006C300121017600202DE0002001900421684696
:208E4000FEF7C8FF250074352868002806D0E06E002803D02800FFF765FC0190042101A8D3
:208E6000FDF79CFE019800283DD0009800283AD001460198814200DD01002800FFF78DFCA4
:208E800031E02100743100200A68002A02D00800FFF748FCFDF7BBFE25E004216846FEF7B1
:208EA00099FF250074352868002815D0E06E002812D02800FFF736FC0099002913D000283A
:208EC0000DD00E46864200DD060031002800FFF764FC0098801B00900098002803D0FE2192
:208EE0000098FDF766FE8C340120207004B070BD03000100080C002008B4024B9C4608BC49
:208F00006047C046F5050020F8B408B40D000799032443009C40E3439024E40526681E4080
:208F2000266026684700BD403543256001258540A6882F00BE43A6806E463678002E02D00B
:208F4000A6883743A780A6681E40A660A668B4466E46377E4600B74066463743A760E668A7
:208F60003340E360E368400082401A43E260002903D0A0690543A56102E0208D054325857B
:208F8000F3BC704759480168802292020A4302609020C005A02189050160C168564A0A4341
:208FA000C26001218161026803239A4351E05348704753480188C806C00F70475048018802
:208FC0004807C00F7047002070474D4800880107C80F70474A4801888807C00F70470120E1
:208FE0007047FF20704766480078012800D0704700B58BE09020C005016830229143016089
:209000000168694A0A4002600CE09020C0050221018501680C22914304222CE09020C0056C
:209020000221816101680C2291430160704770477047704770479020C0051021018503E0BD
:209040009020C005102181610168574A0A4080214900114301607047704770479020C005FB
:209060000421018503E09020C0050421816101683022914310220A430260704780B5FFF794
:20908000EDFFFFF7F0FF01BD52484068704710B50100504C616010D00020206038480078AD
:2090A00001280AD14C4A914204D24C4801F0FCFA001F01E00020C043206010BD10B582B08B
:2090C000040008004349096800912100FEF788FB002016BD2A490978012901D8182100E05A
:2090E000302181803E490160704700001410024070473C487047000055555541E40C0000F7
:2091000010000048012800D0704700B583B000200190032000900023002201210220FFF77C
:20912000F3FE01200190032000900023012200210420FFF7E9FE01200190032000900023E9
:2091400001220021FFF7E0FE01200190032000900023012200210120FFF7D6FE03B000BDD0
:2091600072B601F0E1FB2048022101601F48FFF7C3FE1F48016889B21E4A0A430260FEE7E9
:209180005B1B0020002806D0401E032806D90938022803D904E00948007870470020704751
:2091A0000020C04370470000FFFCFFFF7047002802D111480121018070470000541B0020E8
:2091C000002802D10D48012101607047704770470B487047EC0A002080841E00808D5B00ED
:2091E000006CDC02102700004060004020A107000CED00E00700FA05280000481800004897
:20920000FF3F00200020704780B501228921684600F03CF868460078012803D068460078FD
:20922000FF2801D1002002BD012002BD0120C0437047FEE708B4024B9C4608BC6047C0465A
:209240001F05002008B4024B9C4608BC6047C0469F03002080B57348002101600120FDF725
:20926000CAFC6420FDF735FB72B66F484178491C41706A486A490160FFF772FF01BD6B4834
:209280000178002901D16A4810307047F0B506000C001500002E1ED0002D1CD06019654989
:2092A000884218D2C80884420FD2001B2F00854200D907003A00604821183000FFF71EF93A
:2092C000F619ED1BE419002D05D02A005A4821183000FFF713F9F0BD80B55748FFF7AAFF21
:2092E000002002BDF0B5C1B00C00150000280AD0002D47D0070080200001844203D2601956
:209300004C49884202D30020C0433CE0FF2C1ED880204000061B864200D90600AE4200D948
:209320002E00320039006846FFF7E8F800233200694641482018FFF785FFBF19AD1BA41974
:20934000FF2C02D8002DE3D11CE0002D1AD0FF20C0432418FF20801C854201D3461E00E01C
:209360002E00320039006846FFF7C8F800233200694632482018FFF765FFBF19AD1BA41983
:20938000002DE7D1002041B0F0BD38B5040007D0002901D1002032BD80252D01A94202D0C8
:2093A0000020C04332BD2448FFF744FF2A0000212000FFF797FF32BD002800D1704710B59B
:2093C000002A0FD08B18FF24A41CA3420AD2631E994207D25B1A9A4200D91A00184BC91880
:2093E000FFF78CF810BD10B5C0B080246400A14201D1002802D10020C0430BE02200010008
:209400006846FFF77BF80023220069460C48FFF719FF002040B010BD0000000000010020E1
:209420002143341244120020B8010020B8110020004900080108000000400008004100085F
:20944000003F0008F9B583B00D001700C100081AC000B0490E18B04C2000A4300090806995
:209460008047B079012801D1022496E0E41D0294E0788007800F022800D08DE03069002838
:209480000FD1707EC107C90F684601710A980A90002D45D1002F43D1002843D1706A00283E
:2094A00001D0032479E00024012500212D193A1B0020029B1B78002B06D0049B002B02D167
:2094C0000A9B002B00D0012072613561B176F07600990988491C009B19803181317E002988
:2094E0000DD13188914202DA002800D00A0029000398009B1B69DB6A9847012030760A98B4
:2095000002284BDA049800283BD00146039801F02FFA002838D00021039800F01CFE33E028
:20952000002F02D16846012101713A00290030001C3000F03CF90400381B04D00A980128ED
:2095400015D1002C17D068460079002826D0306A716A401A3188884220D302200A900021AB
:2095600068460079002819D000220025A0E7002102289BD1F4E701213088B84296D2070010
:2095800094E7039801F0EDF970693C1A0298C0788007800F022801D00024E4430098C069C0
:2095A0008047200005B0F0BD18B401001C31C47E641E012C05DB0A0008320CCA0CC1641E0E
:2095C000F9D1C17E491EC17611BC704738B50C00456B04E0A96820006A6890472D68002D37
:2095E000F8D131BD7047FEB584B007000020C04301904948B43000680090002646480078C2
:20960000062859D269460872C100081AC00041490D180098C36C0C980C90180005D00C9ADC
:209620006846017C3800984705E06846017C3800009A5268904704003ED0FF2C3CD03822D2
:2096400000212800FCF752FFF901214369716846007C28716846007A00994969884706003A
:20966000002F03D10C98B04200D806000098026C100002D001A90520904700F0F7FCC2B28E
:209680006846017C300000F0BAFC28806846808A6880002F02D00198E86003E00698E861D5
:2096A0000C9828621C4800780600401C1A4908706000C019A5490E54300007B0F0BD4106FF
:2096C00001D1002070470107C90E000600D5491C9E48405C7047C100081AC0009C490818E1
:2096E000407970476D48817A8807C00F7047F8B5094FB4203C580125954E03E03000A168A3
:2097000088476D1C383638788542F7DBE0688047F1BD00001C0E00206C0F0020F8B55F4C40
:20972000607A00282CD10020C0430090F82200212000FCF7DBFE01272770854DA8225200A3
:2097400000212800FCF7D2FE01F0FAF801F060F92000EC300168002901D1B24901602600AE
:20976000B436002031684969884728803068026C100002D06946052090470098E8606772D1
:20978000F1BD38B5454CB4202558286880472A6C100007D0E11D0620904721000831022001
:2097A0002A6C90471020A0722869804731BDF2B504001500002621E0002924D0E06841180F
:2097C00062688A4200D90A00171AAF4200D92F003A00216809180098FEF790FEED1BA068D7
:2097E000C01BA060F6190098C0190090E068C019E0606168884201D10020E060A168002D22
:20980000DAD1002901D10020E0603000F2BDF2B5040015006068A168461A1CE0E068A16825
:2098200040186168884200D3401A4219914200D911000F1AAF4200D92F003A000099236878
:209840001818FEF75BFEED1BA068C019A0600098C0190090F61B002DE0D13000F2BD10B50D
:2098600000F0AFFC80B500F0B2FC10B582B0002B02D50224002300E0012400F0A4FC80B56E
:20988000334BD86119620120D8761A760020D882B349B4310968096B884701BD6C0F00202F
:2098A000F7B504001F00AE4EB07A8007800F022801D0002008E0E000001BC00024490D184D
:2098C000A879002802D00220C0433DE0A436B0698047E87E00281FD0C100691814314A68BB
:2098E0000B689B18019CA34204D10298101848602F7625E0032802D10324E44321E0083151
:209900000C6002984860E87E401CE8762F763088401C3080288113E029001C3101980860FD
:20992000029848600120E8762F763088401C308028812869002803D120003169096B8847CA
:209940000024F0698047200003B0F0BD681000201C0E0020F2B582B00400E000001BC000C9
:2099600080490E187E4D2800BC300190006800277179090631D500970025804730690028B6
:2099800002D1F07E002820D0B7760298002819D00146200000F0ECFF002816D03069022883
:2099A00000DB451E30001C30F17E012905DB4268AD180830491E0129F9DA0021200000F038
:2099C000CAFB02E0200000F0CCFF019840688047002D23D00120009020E0804730690028A4
:2099E00018D0029800280BD00146200000F0C0FF002808D00021200000F0ADFB012702E0E9
:209A0000200000F0AEFFA87A8007800F022801D00027FF430198406880470097009803B003
:209A2000F0BD0000E5950008F8B504000F00E000001BC0004B490D1800264948BC30009090
:209A400000688047E87E032814D3002F01D5012610E00120A876002F07D03900200000F0B5
:209A600087FF002804D0012602E0200000F079FF0020A8760098406880473000F2BDFEB5FC
:209A800004000F001500089E002E02D5FFF708FF4EE06846037A2A0039002000FFF700FF25
:209AA0000321C943884206D131002000FFF7BCFF0028EED03BE000283AD401960027E000FE
:209AC000001BC00027490E182548BC300090006880473069002802D1F07E002820D0B776B6
:209AE0000198002819D00146200000F041FF002816D03069022800DB471E30001C30F17E29
:209B0000012905DB4268BF180830491E0129F9DA0021200000F01FFB02E0200000F021FFC1
:209B2000009840688047AF4201D2E81B00E0002003B0F0BD42001018C000094A10180163EE
:209B4000704707490A00A6321378032B06D29B00C918A83108601078401C107070470000B3
:209B60006C0F00201C0E0020F2B582B006001500F000801BC000AF490C18002E12D1002470
:209B80009E4E3700A6373878844261DAA0003018A8300268100002D0290002989047641CEE
:209BA000E4B2F0E7E068002803D029000298E268904701200090206900282CD061698D421A
:209BC00001D22F0000E06769002F0DD03A000299FEF794FCED1B0298C01902902069C019FE
:209BE00020616069C01B60616069002802D0A07E002810D0300000F0ADFE00272761607E3E
:209C0000C00706D430007D49B4310968896A8847277609200090002D16D02A000299200047
:209C20001C30FFF7F4FD617EC90702D5218888420AD2207E002807D030007049B431096840
:209C4000896A88470020207600992000FFF7BEFC03B0F0BDF8B50600F000801BC000754907
:209C60000D18E87E002875D0002E02D02869002870D1002068762F001C377868002805D194
:209C8000E87E022802D32800FFF78EFC5B48B43003681C6D20001AD0E88A00906B463A0045
:209CA000E97E3000A04704000098E882601C2861260003E0361A2800FFF776FC7868B04260
:209CC000F8D3801B78603868801938601FE07C682888844200D90400601C28612200396877
:209CE00030005B6B98477868001B7860386800193860002C03D02988481E204001D0002004
:209D000010E0EE8A200000F0CFFC3018E882A88A002808D0E98A002905D02A885143401E07
:209D2000084000D1E8827868002813D1E87E022803D32800FFF738FCF1BD002C08D0E88AD8
:209D4000002805D0287E002802D000202876F1BD0020E876F1BD38B50400E000001BC00022
:209D600034490D18002C0DD0286902280ADB0020C04328610421687E002800D10621280099
:209D8000FFF724FC00202861E87E00280CD02000FFF760FFE87E032818D2A87E002815D077
:209DA000200000F0D7FD31BD20001449B4310968896B8847002C07D0200000F0CBFD4021FF
:209DC0002800FFF703FC31BD01F044F931BD80B5C200121AD200174B9A189171074AB4321A
:209DE0001268126A904701BD80B50121FFF7EFFF01BD0249B4310860704700006C0F0020F5
:209E000070B504000E0015000C220021FCF76EFB6660A560A44801680A0000E01268002A9D
:209E200003D0A242FAD1012070BD21600460002070BD00001C0E002010B4C400201AC00054
:209E40009A4C20184A608B60426B0A60416310BC704710B59648817A002101730122934BDD
:209E60003E3302E01970521C38330478A242F9DB817A102001400820084300F014F810BD51
:209E80008B48807A704780B58948817A0120084300F009F801BD80B58548817AFE200840BF
:209EA00000F001F801BDF0B583B00700804EB47AB42030580190BC4248D0A00719D4B807CA
:209EC00017D5012568460570FFF711FC07E000212800FFF77CFF280001F000FA6D1C307865
:209EE0008542F4D30198026C100002D0694600209047A0070BD5B80709D4684600210170E2
:209F00000198026C100002D06946002090476648046806E06268100002D03900A0689047EE
:209F20002468002CF6D1B772B07A062108420DD0012408E00021200000F00DF9200000F0AD
:209F4000B9F8641CE4B230788442F3DB03B0F0BD01000020564A927A9207920F022A05D195
:209F6000C800401AC00051490818406A704738B505004F4CBC3420688047E800401BC00015
:209F80004A4908180169022901DB4D1E00E0002501001C31C07E012805DB4A68AD180831E8
:209FA000401E0128F9DA60688047280032BDC100081AC0003D49081840697047C100081A15
:209FC000C0003A490818C17E002902D00020C0437047C18A828A002A0AD0002906D0038825
:209FE0005943521E0A4008D10021C18200207047481E8041C043C00F70470120704702006D
:020000040800F2
:20A00000032905D14020824213D24008FBD17047402A01D340207047202A01D32020704700
:20A02000102A01D310207047082A01D3082070470020704701700A0A42700A0C8270090E19
:20A04000C17070470170090A417070470178427812020A43817809041143C07800060843B5
:20A0600070470178407800020843704780B51048B4300068806980470221084002BD80B50C
:20A080000B48B430006880698047C007C00F02BD074A5078411C517041000918C900511851
:20A0A0002A31087070470000641000201C0E00206C0F002070B50400E000001BC000474929
:20A0C0000D180026AE716879000604D52E61EE76EE8220210DE06E62AE622E61287E002888
:20A0E00005D020003E49B4310968896A88472E7610212800FFF76AFA200000F02BFC70BD11
:20A10000C200101AC000354A1018C160704778B4010001200024324B1D00C826AE59002EE5
:20A1200005D1A0001818C8300160002003E0641C2D1D052CF1D372BC70472949DC31086092
:20A140007047C200101AC000244A10184279120600D441767047F8B504000F002048B430E5
:20A160000168E000001BC0001C4A1518002C19D000266879000607D52000896B88472E61B8
:20A18000EE76EE82202105E02000896A88472E762E6110212800FFF719FA002F02D020002D
:20A1A00000F0D8FBF1BD0E49EC31086070470C4BB833186059609A6070470949F431086098
:20A1C000704782B000240094FFF73CF916BD032300930023FFF736F902BD00001C0E0020D6
:20A1E0006C0F002080B5006801F04EF901BD7047800700D1704780B500F08EFA01BD30B51B
:20A2000089B0FFF73DFE8007800F022859D1934C2068002855D060689149096A401A01281E
:20A220004FDA2069002804D12000143001F030FA20612169002921D00025ED432B00626980
:20A24000A06801F051FB002818D4A06961694018A0612000143001F01BFA206100280DD089
:20A260002B0062690100A06801F03EFB002805D4A06961694018A06100202061A0690028B6
:20A280000DD0A06801F040FB0500A069401B01F0F1F9A56103E00100684601F048F901F0AE
:20A2A000E0F90500202D02DA002D01D109E020250023DB432A006946A06801F00BFB012828
:20A2C000E9DA09B030BDF0B585B000250027012101A8FDF77FFD04216846FDF77BFDFEF780
:20A2E00093FF0028009804D0FCF7B0FC02AC5D4D51E00830FDF742FE040005D10098FCF73F
:20A30000A5FC02AC012545E00099FDF763FD68460079002806D0022829D00CD3042832D061
:20A320002BD336E02000FCF7C4F80100201D01F0FEF805002FE02000FCF7BBF80600200015
:20A34000FDF742FE30000830FDF718FE040002D102AC01251EE03100083001F027F907002D
:20A360003E483F49096AC2688918416013E02000FCF79FF801F0D4F80DE02000FCF799F805
:20A380003649C86007E02000FCF793F801F07CF801E00225ED4329002000FCF775F8390012
:20A3A000201DFCF771F8083739002000FCF7F6FB02A8844202D02000FDF706FE05B0F0BDCC
:20A3C0007CB5264CFEF720FF012141402160FEF719FF002804D1206800283BD001F09DFB54
:20A3E0002068002836D001AD402000900023002202210120FFF7F7F82870402000902300F0
:20A400001C33002202210020FFF7EDF86870002000900023082203210120FFF7E4F8A870A9
:20A4200001A801F07BFAA0600F4901F045FA0F49A06801F048FA0E4E0023320021005C3193
:20A440006878FFF7F9FC00233200210068312878FFF7F2FC0020E06073BD00005C0A002088
:20A46000B8010020FAFEFFFFE5A10008EFA10008F1A10008554800218170704710B582B0F0
:20A48000009301234000514C205CFFF7F8FA16BDFBB5170040004D490C5C089E002F16D130
:20A4A0002000FFF78BFD0500012D10DA002E04D5002D14D00320C04311E031002000FFF76B
:20A4C00049FA002801D1002DEAD1002007E000966846037A3A0001992000FFF7D0FA03B028
:20A4E000F0BD10B54000394C20184078FFF7B7F910BD80B54000354B18184078FFF7B2F944
:20A5000002BD80B54000314908184078FFF720FD02BD80B540002D49085CFFF728FD02BDBA
:20A5200080B54000294908184078FFF740FD02BDF8B507000124254DA878002804D1AC70E6
:20A54000E8702348FFF7E3FDFFF7A2FD41000818C00020490E182436FF20F07030717071C2
:20A56000387801218140787884400C43348000BF1AA000F0BDFEF071E878410069183A7838
:20A580000A707A784A700978CA00511AC900124A5118802212018A82411CE970F2BD80B5F6
:20A5A00040000A4A10184078FFF7AAFD01BD80B54000064A105CFFF7CDF902BD80B54000AB
:20A5C000024A105CFFF730FA02BD00004E1B002075A400086C0F00201C0E002042554C4B27
:20A5E00020696E746572666163650000F8B50700002472B60E4D6878401C687004260BE006
:20A60000C068017C314205D0C1682A6A891A012900DA0124FCF7D0F838680028F0D16878A0
:20A62000401E68706878002800D162B62000F2BDB801002030B585B0029001900F4B9C68B0
:20A64000039472B69C68E2601D6A521B012A04DA5878002810D162B60EE0026800926A466D
:20A6600002600098002800D042606846A060042008432074FCF70AF905B030BDB801002024
:20A68000CA0F00D0494203105A400DD004B500D3404200F009F8009AD20701D349421242D7
:20A6A00000D5404204BD0000094210D088420BD30122002300185B418B4200D35B1A52410D
:20A6C000F8D319001000704701000020704708B501F03CFA08BDFEE7204C200000F0B6F83F
:20A6E000FCF7ECFF0500FFF78AFD00F089FF200000F0CCF8002DF0D0012120001030FDF74B
:20A70000E3FBEAE780B5154800F0C0F801BD80B5124800F09BF801BD80B510481030FDF701
:20A72000ADFB01BD10B584B00C4C200000F079F802212000103001F00BFA02200290400272
:20A740000190200018300090054B012205A18320C000201801F014FA04B010BD0006002016
:20A76000D9A6000842475461736B0000F8B572B61B482830C0C81948C068804704000025A5
:20A78000164800698047002806D00020761C47411248C06880470400104842690023007A06
:20A7A000002804D10021101BA94104000D003000390001F01DFA00196941084A92690023B1
:20A7C00001F016FA054AD269002301F02AFA044A5278002A00D162B6F2BD0000980B002019
:20A7E000B8010020F8B5070030480468304D012614E0207A002810D06068B8420DD1267276
:20A800002878401C2870207A401E2072000602D1200001F03BFAFBF7B6FFE468002CE8D123
:20A82000F1BD10B50400234823490160102200212000FBF75BFE72B61C480168E160046011
:20A840001B484078002800D162B610BD38B50400174D2878401C2870A868217A002902D16F
:20A86000606001250DE06168814208D01021200001F01EFA207A0028F8D1A8686060257A4D
:20A880006D1C2572FBF77FFF280032BD80B508490A78521C0A70017A491E0172090601D1EB
:20A8A00001F0F4F9FBF76FFF01BD0000880B0020B8010020900B0020E5A7000812420FD08E
:20A8C000814202D25318984203D310B5FDF716FE08BD80185B1E1978401E0170521EF9D189
:20A8E000704718B402E0401C491C521E002A09D00B7804789C42F6D002D20020C04302E043
:20A90000012000E0002012BC7047FEE700B58022520009495005FDF705FE08480168032287
:20A920000A430260002000BD04480168032291430160002070470000004800080000014014
:20A9400038B5174C06252000FDF7BCF808346D1EF9D131BD80B5C0001149081801F0C2F91A
:20A9600001BD80B5C0000E49081801F0D7F901BD80B5491CC0000A4A1018FDF7A5FA02BD06
:20A9800008484178491E41704078002800D162B6704772B603484178491C4170704700001D
:20A9A00088100020B801002035480168802292020A43026033480168334A0A4002600168C5
:20A9C000BB2212030A43026030480168C20B0A43026070472D4801682D4A0A40026070470A
:20A9E00030B42C490860802000062B492B4A13680B40034313601368C02424061568294019
:20AA00001B191C400C4314602549086030BC704780B524480168244A0A400260C16880227B
:20AA200012040A43C26019480168194A0A4002601E48FFF7DEF91E4A1E491F48FFF7B7FBA7
:20AA40001E48FFF7B0FB1E48FFF777FB01BD10B51C4C2078401C20700E480068010000D023
:20AA6000804772B62078012804D16068002801D0FCF7F9FF2078401E207062B610BD00003A
:20AA80001410024004080140FF0FF0FF585C0040FF7FFFFFC40C0020FFFFFF001CE400E0C9
:20AAA00000E100E010100240FFFF7FFFA0F8000881A9000893A90008E1A90008A9A90008F5
:20AAC000D5A90008B8010020026843689A4204D2836899540168491C0160704738B50400A1
:20AAE0000D00C9B2FFF7F0FF290A2000FFF7ECFF31BD000030B583B0002812D100909F482D
:20AB0000029080204000019004216846FFF7DCFF03216846FFF7D8FF99496846FFF7DEFF8C
:20AB200050E0012812D016D3032805D009D3042811D100BF25A51FE09248E0304069C568BF
:20AB40001AE09048E0304069856815E08D48E0304069456810E08B49052807D3401F8A7B1E
:20AB6000904203D280000818056905E0E03109680A0003D088470500002D01D1002022E0E7
:20AB800028000021002401E0401C641C0278002AFAD1009179480290802040000190610066
:20ABA000891CC9B26846FFF78FFF03216846FFF78BFF002C06D029786846FFF78FFF6D1C93
:20ABC000641EF8D16D4803B030BD0000436F6E66696775726174696F6E00000080B5012225
:20ABE00000210120FEF74BFE01BD38B56549B4228C588278C3781B02134347D18279C379CB
:20AC00001B021343022B41D1491C03234A7A520707D40078184239D10B7B58480370022266
:20AC20001DE002224D7A154205780FD12B4013D0022B04D03CD20079002827D102E0007927
:20AC4000002823D14D48002202802EE02B4003D0022B16D009D324E00B7B48480370897AD4
:20AC600011421ED01A4302701BE00978491E0079814202DA606A804713E04048002101702B
:20AC80000FE00079FEF71BFDFF2802D1606A804731BDC100081AC0008E49081880793749B3
:20ACA000087036480021417000220221FEF7E7FD31BDF8B502000C003248B4300568907832
:20ACC000D17809020143E6B21079032952DA9379D7793F021F434DD12A4B0A33012909D190
:20ACE000002C587802D00221014301E0FD21014059703CE01F787F073CD503271B789B076D
:20AD0000127814D4174002D0022F03D032E0022930D12CE000292DD1FEF7D1FC002829D13F
:20AD2000601E8041C043C00F6A4988711FE0174002D0022F03D01DE000291BD117E00028F9
:20AD400018D0802816D0FEF7BAFC0400FF2C11D03100FFF73CF8002E09D1200000F0BEFA97
:20AD600000212000FFF7F7F92000FFF7A3F9FFF735FFF1BD686A8047F1BD0000B8100020F3
:20AD8000090400006C0F0020F4B582B005000E00108840080024002803E0C10700D5641CF1
:20ADA0004008FAD109212800FFF78EFE04212800FFF78AFEF1B22800FFF786FE0298817809
:20ADC0002800FFF781FEE1B22800FFF77DFE0298C1782800FFF778FE029801792800FFF711
:20ADE00073FE029841792800FFF76EFE0298C1792800FFF769FE02988268100002D029001C
:20AE0000300090470124334F3C37A048B430009006E00126F1B22800FFF756FE641C3837A4
:20AE20009A480078844253DA029800880121A1400842F3D007212800FFF746FE05212800BB
:20AE4000FFF742FE79782800FFF73EFE39782800FFF73AFE3E1FFFF712F9002803D10022EE
:20AE60003978308807E0E0B200990968496988470122397880B2FFF7C2F83080318828001E
:20AE8000FFF72CFEE000001BC000124908180179012902D0032906D0BBE74688112E15DA46
:20AEA000002EB7D1B5E74688FFF7E9F8002807D1FF2E01DDFF26ADE7002EABD10826A9E76F
:20AEC000112E03DA002EA5D10426A3E71026A1E703B0F0BD1C0E0020F0B585B080246B4865
:20AEE000401C0090807AC00700D5A0240098007B002802D0200040240443002001906448D7
:20AF00000390802040000290092101A8FFF7DCFD022101A8FFF7D8FD002101A8FFF7DEFD58
:20AF20000098017801A8FFF7CFFD012101A8FFF7CBFD042101A8FFF7C7FD210001A8FFF7C4
:20AF4000C3FD5448017801A8FFF7BEFD00254F4F11E06C20305CA84205D132007032290039
:20AF600001A8FFF711FF641C1C36009840788442EFDB6D1C183700980078854211DA43484B
:20AF8000C4300268002A03D001A92800526890473A002432290001A8FFF7F6FE00243B4EFA
:20AFA000E3E701993A48801CFFF74CF8384805B0F0BDF0B583B000200090354F02978026A8
:20AFC0007600019612216846FFF77EFD01216846FFF77AFD71006846FFF780FD2B4C251D8A
:20AFE00029786846FFF770FD69786846FFF76CFDA9786846FFF768FDB7480188C9B26846D6
:20B00000FFF762FDE434206901886846FFF766FD206941886846FFF761FD2068010002D0FB
:20B020008047010000E031006846FFF757FD01216846FFF749FD02216846FFF745FD032106
:20B040006846FFF741FD01216846FFF73DFD380003B0F0BD38B50D490C000A34A0780006CB
:20B0600013D5A0784006400EA070A5782800B4310968C9698847002D217802D00420084389
:20B0800001E0FB200840FEF70EFF31BD6C0F0020B81000201C030020F0B583B005009B4CF6
:20B0A0006678002E0DD02700380024304169080004D028008847002800D10AE11837761EB0
:20B0C000F2D12000B430019001680E0028786022024006D0202A00D1D8E0402A00D1E6E093
:20B0E000F5E068780B2800D9F1E002A2125C5200974400BF060AED0CED112FED676F849BA8
:20B100002800FFF772FDE4E0002100E001212800FFF7CFFDDDE0AD78207A002813D0280022
:20B12000C9698847002DA17A02D00420084301E0FB200840FEF7B7FE207A012800D0C8E05C
:20B14000FFF74CFDC5E0FFF749FD802028432073BFE000260024E8790002AF7907436846C5
:20B1600001210170E878012810D012D3032801D004D30EE0A878FFF7BDFC09E0FFF7ACFED5
:20B180000400801CFEF76DFF060002E0FFF711FF0400002C03D101980068406A98E0002E6B
:20B1A00000D12678BE4200D93E00BE4202D16846002101706846027831002000FEF75FFB2E
:20B1C00087E0FEF78FFA6946087000220121684626E0A878012805D1FFF700FDA17A02201C
:20B1E000084306E0002807D1FFF7F8FCA17AFD200840FEF758FE6CE0486A69E0A8780028DA
:20B2000011D1A87901280ED1A07A06220240062A01D0486A5CE0684600210170002201212C
:20B22000FEF72DFB55E0486A52E028790190A07A06220240062A27D16078019A904223DBB7
:20B24000A878EA78170207438020400087421BD2FFF7C4FC01250BE0EEB200213000FEF7C6
:20B26000B6FD300000F03AF83000FEF723FF6D1C20788542F0DBF0342268100029D03900DF
:20B280000198C0B2904724E0486A21E02879617888421CD241000818C00020182430C1680D
:20B2A000080014D028008847002810D111E02879617888420BD241000818C00020182430E3
:20B2C0000169080003D028008847002801D0706A804703B0F0BD00001C0E00200B49B431B5
:20B2E0000968C96B0A0000D1704780B5884701BD064A937B052B01D300207047591C9173A3
:20B300009900511808615B1DD8B270476C0F0020F3B504006668A068801B01D52169401899
:20B320000090904200DB0092009800281DD00546206921680818801B2F00854200DD07009F
:20B340003A0031000198FDF7D9F80198C0190190F619ED1B2068216941188E4200D10600F8
:20B36000002DE5D16660E6600098F6BDF3B504001500A6686068801B401E01D5216940184B
:20B380000090A84200DB0095206921680818801B2F00854200DD07003A0001993000FDF724
:20B3A000ADF8F6190198C0190190ED1B2068216941188E4200D10600002DE5D1A66000983B
:20B3C000F6BD10B582B08D4C6078002817D02079A179014313D100202063606301226946F0
:20B3E00020001C30FFF794FF012808D1A748006A2063012020716846007800F0D4FC13BD12
:20B4000038B505007D4CA148006A20636078002803D000F095FD002809D1012229002000D8
:20B420001C30FFF775FF002801D0002032BD00202071012032BD10B57049944A126A4A6308
:20B440000B69CA68D21A521E01D58C691219002A0BD018700869401C8B68FF24A41C1C198F
:20B46000A04200D118000861521E487800280AD0C878002807D1022A05DA086C002802D1AC
:20B48000012000F04DFD10BD70B505005B4C2078002818D100F034FDA0700020E070FF2644
:20B4A000B61C3000FCF76AFDA060E06020616061A6618120FCF762FDE0612062606281208E
:20B4C000E06201202070E069002813D0A068002810D0E06B85420AD0A06B002801D0401EC7
:20B4E000A0637A4B7A4A7B49280000F06CFCA06B401CA063002020636063A07860700120A3
:20B500006071E56370BD10B5734CA06B002806D0401EA06303D100F0D5FC0020E06310BD32
:20B5200072B66D490122CA70086462B67047F8B5324CA26B002A36D00A00010020001C30B6
:20B54000FFF714FF0500012D2EDB0127A77100262079002823D16079002807D0667100F0EC
:20B56000EFFC01281DD1667000F0E3FC6078002803D000F0E5FC002811D126636663012201
:20B58000694620001C30FFF7C3FE012807D13F48006A206327716846007800F004FCA6719F
:20B5A00002E06770E5E700252800F2BD38B54A4CA26B002A1DD06269E3689A4201D0002080
:20B5C00032BD0A00010020000830FFF7A1FE0500607800280ED0E07800280BD1002D09D03F
:20B5E000206C002806D0002000F09AFC0020206400E00025280032BD000000001C0C002013
:20B6000070B582B00126344CA67100252079002823D16079002807D0657100F091FC0128E7
:20B620001DD1657000F085FC6078002803D000F087FC002811D12563656301226946200044
:20B640001C30FFF765FE012807D11048006A206326716846007800F0A6FBA57173BD667095
:20B66000E5E71D49086A4A6A801A401E01D5C96A401870471849CA6810188A698B689B180E
:20B68000984201D35342C018C8607047B801002078B40100104A53691069984202D2906974
:20B6A00095682818C41A0AD018001B19956996687619B34201D36E429B19536100E00020DD
:20B6C000002900D00C6072BC70470000C3B3000837B4000801B400081C0C002070B5040081
:20B6E000874D286E002820D44200101800012E18072903D00020FEF777FB0EE02000FEF786
:20B70000A5FC70602079307260797072A079B072F168080001D0301D88470020C043286688
:20B72000012200210120FEF7AAF870BD38B502794179090211430023714A1400143401E044
:20B740005B1C30346F4D2D78AB4203DA25888D42F6D103E00023DB43002D43D45900C918FE
:20B76000090154184178202906D03BD3222918D004D3232926D035E0136631E0251D2968AF
:20B7800020002630FEF756FC20002A302979017069794170A97981700022072126342000F5
:20B7A0001CE0241DE168002915D069468278D307DB0F0B7080788207D20F4A706846E168FA
:20B7C000884708E0241DE1690A0004D0C2781202807810438847012200210120FEF74FF840
:20B7E000002032BD012032BD70B50C00002244490B001433434D2D7801E0521C3033AA4225
:20B8000003DA1E888642F8D101E00022D2435000801800010D1805212000FFF755F924211F
:20B820002000FFF751F900212000FFF74DF9882149002000FFF752F905212000FFF744F95F
:20B8400024212000FFF740F901212000FFF73CF903212000FFF738F9A98CC9B22000FFF7B6
:20B8600033F904212000FFF72FF924212000FFF72BF902212000FFF727F906212000FFF724
:20B8800023F905212000FFF71FF924212000FFF71BF906212000FFF717F9A98AC9B22000AE
:20B8A000FFF712F9A98CC9B22000FFF70DF970BD1448002141707047420010180001604A94
:20B8C0001018C16070474200101800015C4A10180161704710B5440020180001584C2018F8
:20B8E0004078FDF7C2FF10BD10B582B000930123440020180001524C205CFEF7C0F816BD49
:20B90000600C0020581B002080B54100081800014B49085CFEF72BFB02BD0000F1B582B0C7
:20B92000012448484078002810D146484470444D602200212800FAF7D9FD42480021017010
:20B940000020C04328664048FEF7E1FB3F48FEF7F8F8FEF79DFB050001953D49FEF7EAF8EC
:20B960003C4F68004019C0003D1824353A48A8600220E87028716C7102988078012181401E
:20B98000298036A0FFF7B4FCE871FEF781FB050068004019C0003E1824360020B0600A2028
:20B9A000F07000203071707102980078012181400298407884400C43348000BF28A0FFF7FA
:20B9C00097FCF071C4203C58002C09D0002000900023022202210198C0B22468A04705E079
:20B9E0003F1D0220387000207870B8701548007841000818000112490C1802980078207099
:20BA000002984078607002988078A07001216078FEF797FB221D00BF19A003C803C2019801
:20BA2000A082A5840A2200BF12A116342000FCF765FD04480078411C024A117003B0F0BD10
:20BA4000600C0020581B0020B1B80008DDB600082DB700086C0F0020E9B7000843444300C2
:20BA6000434443204441544120696E746572666163650000A120000000000200000000002E
:20BA800000C2010000000800F8B4059C2D4D2E78761C2E70F6B2042E08D2B700BE19AD1936
:20BAA0006D1E2871E9702A70AC706B70F1BC704738B50C000021234D2D1D2A79824227D1E1
:20BAC00008212000FFF700F80B212000FEF7FCFF29792000FEF7F8FFE9782000FEF7F4FFDC
:20BAE00029782000FEF7F0FF69782000FEF7ECFFA9782000FEF7E8FF287941000818C000E1
:20BB0000114908182B3001782000FEF7DDFF31BD491C6D1D0329D0DB31BD10B5094C0F22F9
:20BB2000FF21201DFAF7E2FC002020700648C42114344450001DEF21017002214170012186
:20BB4000817010BD000300206C0F00207047FEE770B504000E0072B6084D6878401C687005
:20BB6000082200212000FAF7C1FC66716878401E68706878002800D162B670BDB8010020C8
:20BB8000FEB506000D000A9F44220021FAF7AEFC341D01982061207B134909780143217359
:20BBA00039203754002D00D02562089FA762099D65622A00CD213800FAF798FC7819072172
:20BBC0008843503800210160802149044164074901640299C1640221C94341622060300006
:20BBE000FAF728FE03B0F0BD571B00201F7A000830B4434351435D18010C0C00130C5C4351
:20BC00002D1980B2434392B251430024C918644124040B04090C09195043C018694130BC35
:20BC20007047124224D0994228D970B500251B4202D00C00002109E0002401264918644149
:20BC4000944200D3A41A7641F8D33100012601E0764109D2001864416D41A41A9D41F7D260
:20BC6000A4185D41B619F5D3300022002B0070BD1B42D8D108B500F08BF908BD01D1904289
:20BC8000D3D202000B0000210020704710B5040002E0C068FAF790FD72B620680028F8D108
:20BCA00002484078002800D162B610BDB801002000B585B002900190094A9368039372B6B2
:20BCC000036800936B4603600098002800D0436090686A4682600174FAF7D8FD05B000BDE8
:20BCE000B801002038B504000B4D2878401C287072B66878401C68702000FCF7BFF8200068
:20BD000000F048F96878401E68706878002800D162B6FAF738FD31BDB801002038B504000D
:20BD200072B60E4D6878401C68702079002807D148212000FFF7BCFF6079022805D102E0DE
:20BD40006079012801D0002020716878401E68706878002800D162B631BD00BFB8010020D2
:20BD600038B57A4CE5690F202062A80604D5A08CC0B2774949688847280613D5684674492B
:20BD80008968884700280AD020688021884320609020C00501686F4A0A40026031BD68468E
:20BDA0000078208531BD9021C9050A68694B1340802212031A430A606449088508688022B6
:20BDC00002430A607047F2B5050017001E00604C2078002801D000F075F8E66067600098DD
:20BDE000A0605D480168802292020A4302609021C905CA68594B13408422D2021A43CA60A7
:20BE00008A68574B13438B604A6A564B13404B624A6A88235B0013434B620A68524B1340D9
:20BE20000B608022D2038A610A68504B1340820C1A430A600A68474B13400B600A684C4BB5
:20BE40001340802292031A430A600126C1693143C1614168B2030A4342603C4F002038601A
:20BE60007860B860F00338604248854200D3451EE80F40194010404940182900FEF700FC25
:20BE8000082801D2082003E03104884200D3481E3A4A02400007400F1043B88138680D21E6
:20BEA00001433960364801680902090AB2070A4302603448F10601603868202101433960A6
:20BEC0002670F1BD24480168802292020A4302609020C0050168244A0A4002600168234A96
:20BEE0000A40026001681B4A0A4002600168204A0A4002600020154908601549087070472A
:20BF000080B5012288216846FDF7C0F968460078FF2803D068460078012800D0002002BDA7
:20BF20001A49002801D0402001E08020C003086070479020C00501680C4A0A40026070474B
:20BF4000114800880006C00F7047000000380140100B0020FFFFF3FF14100240FF0FC3FF9A
:20BF600000F03C000FF0FFFFFF3FFFFFFFCFFFFFFFFFCFFF41420F0000D8B805F0FF0000AE
:20BF800018E400E000E100E010000048180000487047FEE772B600210171034840780028CA
:20BFA00000D162B6704700BFB801002008B4024B9C4608BC6047C046F905002010B5FDF716
:20BFC0005EF904007020FAF71CFE70212000FAF7E5FD10BD7047F0B585B0070068460021B3
:20BFE00001700020C043FBF7A5FB03ACCD2F06D1022103A8FAF720FE2078617805E0032142
:020000040800F2
:20C0000003A8FAF719FE6078A1780902401880B2C01D0490C6107400601CFBF7AFFF02907E
:20C0200080190190029800280CD12000FAF70EFE3000FAF7D5FD6846062101700121FAF7CE
:20C04000ADFD4CE031000198FAF7F6FD31000298FAF70EFE0024FAF72BFE311A0D1B0028BB
:20C0600003D0FF2DF7DD3F208543EB00B14204D104984007400FC01F1B1868460078002881
:20C080000DD1B3480078012810D101980219011902980019FDF712F86946087006E0DB1DC1
:20C0A000DA10002101980019FAF720FAD52F13D02900CF2F0CD1A7484078002808D06019AD
:20C0C000B04205D1019800196A4612784255491C01980019FAF789FD6419B442BBD19D4C9F
:20C0E0002078002802D1684600782070D52F0AD0FAF79CFDCF2F06D16078002803D1684638
:20C100000078FAF778FD0298FBF75EFF05B0F0BDF0B583B0032101A8FAF78EFD01A80578AF
:20C120004178807800020C1801202907090F884040100090661C3000FBF720FF070009D173
:20C140002000FAF783FD2000FAF74AFD0620FAF752FD3BE0281126D121003800FAF788FD76
:20C160000026FAF7A5FD211A8D1B002803D0FF2DF7DD3F2085430098002803D06843800A39
:20C18000FAF7A7FB29007019A04203D1B81900224255491CB819FAF728FD7619A642E0D1A6
:20C1A000FAF744FD0FE021003800FAF745FD0098002802D06043FFF7F9FE002038553100D2
:20C1C0003800FAF7EBFC3800FBF7FEFE03B0F0BD1CB56C46FCF7EBFE208000F06FFFA0705C
:20C1E00000F070FFE07000F071FF207100F073FF607100F074FFA07100F075FFE07108211A
:20C200006846FAF7CBFC13BD80B50420FAF7F9FC9848FAF7F6FC80200001FAF7F2FC01BDA8
:20C2200080B5042101A0FAF7B9FC01BD335AEAB800B589B0202200216846FAF757F9C8491F
:20C240006846FAF721F968461C2101717C214171A12181710221C1712021FAF79FFC09B0EA
:20C2600000BD00B583B06846FCF734FF06216846FAF794FC03B000BD80B5FCF73AFFFAF72D
:20C28000C6FC01BDF0B5A3B0002700260025042101A8FAF7D1FC12E0400040100090FA21FB
:20C2A00089000098201AFAF752F904002000A90002AA50506D1C761C0198400801900198A8
:20C2C00000281BD0C007F6D50D2E03D10220FCF759FFECE73000FCF755FF0400B01E0228F7
:20C2E00002D919380128E1D8042280216846FCF7CDFF00980028CFD50097D0E7A90002A8F7
:20C30000FAF74CFC23B0F0BD70B5A2B00024002504216846FAF790FC92480021C94301AE9E
:20C320000DE0D20706D50A00042C00DA0268AB00F2506D1C641C009A52080092001D009AAB
:20C34000002AEED1A90001A8FAF728FC22B070BD5B1B0020521B002000B583B0042101A8B5
:20C36000FAF76AFC04216846FAF766FC0198002808D10078FAF73FFC0198401C01900098E4
:20C38000401E00900098002803D001460198FAF705FC03B000BD80B5FBF7E1FDFAF737FCB1
:20C3A00001BD10B5C0B080246400220000216846FDF702F872E0F0B585B00024E443802785
:20C3C0007F003800FBF7DAFD050004D186204000FAF73CFC49E03900FAF72EFC042102A8A8
:20C3E000FAF72AFC082103A8FAF726FC00223900280000F07DFE0299884236D1082203A90F
:20C400005948FAF761F800282FD100242E000122210001A8FCF7D0FF3078694609790140EE
:20C42000814220D1641C761CBC42F0D328002030FAF73FF8002816D02800FAF73AF8040078
:20C4400011D0042200216846FCF7B6FF00980021C943884201D0844205D139002800FCF70E
:20C46000C2FF040001D50024E4432000FAF7CFFB05B0F0BDE32E000080B580204000FAF782
:20C48000E5FB0020FAF7B7FB01BD10B5C0B080246400220000216846FCF7F8FE2100684655
:20C4A000FAF77CFB40B010BD10B5040004222021FCF7ECFE0422242120000830FCF7E6FEB0
:20C4C0000422402120000C30FCF7E0FE0422482110342000FCF7DAFE10BDF0B589B000251A
:20C4E000ED43802636013000FBF748FD040003D1BE48FAF7ABFB2DE032000021FCF7C6FE3C
:20C50000F70839002000FAF797FB04216846FAF793FB082101A8FAF78FFB00223900200026
:20C5200000F0E6FD0099884211D1082201A90E48F9F7CAFF00280AD103A8FFF7B5FF310077
:20C540002000FCF722FF050001D50025ED432000FBF73AFD2800FAF75AFB09B0F0BD00005A
:20C56000335AEAB8D00A0020F0C7000880B580204000FAF76BFB01BDF0B5CBB00027012140
:20C5800002A8FAF759FB6846FAF778FB6846007A002812D06846007A022841D180277F00DE
:20C5A000082103A8FAF748FB082203A990A0F9F78BFF002804D0002013E180273F01EFE726
:20C5C0003800FBF7DBFC0190002801D03E0003E0802676000AA801903800FAF718FB0024F0
:20C5E0003500BE4200D93D006846007A002805D12A0021000198FCF749FE04E02A0021007D
:20C600000198FCF7D9FE29000198FAF7C7FA64197F1BE5D101980AA9884200D1E4E0CDE01E
:20C620006846007A012869D1009880210901884200D0C6E06D48FBF7A1FC040027D0009914
:20C640000C31FAF7F9FA00220099200000F050FD050000982018F9F72CFF854209D10822E6
:20C6600000982118091D00BF61A0F9F72DFF002802D00020C04306E005A8FFF715FF009994
:20C680002000FCF782FEFAF7C2FA200096E005A8FFF70AFFFCF720FE00240025009E802080
:20C6A0004000864200D9060031000AA8FAF7C4FA2A0031000AA800F01BFD05003200210094
:20C6C0000AA8FCF70FFEA4190098801B0090E5D10C210AA8FAF7B0FA0AA8F9F7EAFEA84284
:20C6E00007D108220AA9091D41A0F9F7EDFE002802D0FCF7F1FDFF43380073E06846007AD3
:20C700000328009863D180214900884259D186204000FBF733FC060053D000990C31FAF74D
:20C720008BFA00220099300000F0E2FC050000983018F9F7BEFE854209D10822009831187E
:20C74000091D00BF2AA0F9F7BFFE002802D00020C04330E0009F002435000122210002A86A
:20C76000401CFCF729FE28786946497A014081421FD1641C6D1CBC42EFD330002030F9F704
:20C7800098FE002815D03000F9F793FE040010D00422002101A8FCF70FFE01980021C943AB
:20C7A000884201D0844204D139003000FCF71BFE01E00020C043FAF72AFA3000FBF704FC93
:20C7C00012E000980C30FAF741FA002009E0002801D00C3000E0082000900098FAF736FAD8
:20C7E0000120C043FAF713FA4BB0F0BD0C080000494453454747455200B583B0012101A85E
:20C80000FAF71AFA0090002811D168460079FE2803D0FF2804D1022004E09148007801E025
:20C8200000F096FC009004216846FAF7B7F903B000BD80B502216846FAF7FEF968460088DE
:20C840008849884202D168460021018068460188FA208000484300F0F0FB01BD80B500F000
:20C8600095FC01BD80B500F095FC01BD70B584B0012102A8FAF7E0F904216846FAF7DCF96D
:20C88000042101A8FAF7D8F900283BD400980199014337D0019EFBF762FBB04202D2FBF7AE
:20C8A0005EFB06003000FBF769FB040002D100F02FFA27E03200AA21F9F718FE019D2900D2
:20C8C000B54200D931006D1A6846007A642802D0652806D00BE02000FAF7AEF9002808D53F
:20C8E0000DE0009820602000FAF758F901E000F00FFA002DE3D10098401E0090DED12000C1
:20C90000FBF762FB04B070BD10B582B00124012100A8401CFAF790F901216846FAF78CF9E5
:20C920000220FAF793F9002813D1684640780002694609780843FF21891C884205D0954927
:20C94000884202D09449884200D1944C2000FAF75EF913BD80B504216846FAF76DF968469E
:20C9600081780902C2781143FF22921C914205D0884A914202D0884A914202D10078F9F757
:20C9800007F801BD002086490A3104220B88002B00D0401C1C31521EF8D170470100002042
:20C9A0007F4A0A3213888B4205D0401C1C320428F8DB0020C0437047FFB583B00224784DE0
:20C9C0000027002628000A300188002924D1F000801B80002C18049820600598606068468B
:20C9E000007E20720CA800786072684680896081AF48006AE0606846FAF7C4F8009820617C
:20CA0000019860613000FAF795FEFFF7BBFF012823D1FCF7E8FA20E0761C1C30042ED3DBA8
:20CA2000A348006A002629000C31B74B8A1E1288002A0CD00A68821A9A4208DB3000FBF7DC
:20CA4000D7FDF000801B80002818478103E0761C1C31042EEADB641EB3D107B0F0BD0000CC
:20CA60005B1B0020FFFF000070B59AB0012102A8FAF7E2F8042105A8FAF7DEF8042104A8B2
:20CA8000FAF7DAF8012101A8C01CFAF7D5F8012101A8801CFAF7D0F8022101A8FAF7CCF8CD
:20CAA0006846007A642802D0652829D044E068468088002815D195480188491C0180684688
:20CAC00081808088FFF76AFF0028F4D56846807900906846C379049A05998088FFF76CFF37
:20CAE0002AE068468088FFF759FF002824D4C100081A80002A4908186D49096AC1601BE0CD
:20CB000068468088FFF74AFF040015D4E000001B800023490D1800266E81A869002802D007
:20CB2000FBF752FAAE612000FBF762FDFFF72AFF002801D1FCF75EFA06A8039068468188DB
:20CB400003A8F9F78FFC042103A8F9F78BFC102103A8F9F787FC042103A8F9F783FC0024B6
:20CB60000F4D102229000398FBF7C8FC039810300390641C1C35042CF3DBFCF718FA01006A
:20CB800003A8F9F776FC21010C3106A8FAF706F81AB070BD0103000001060000FF05000086
:20CBA0004812002030B583B0022100A8801CFAF743F8002401AD19E002216846FAF73CF88F
:20CBC000022101A8FAF738F80221A81CFAF734F80221281DFAF730F80221A81DFAF72CF8E6
:20CBE00001A96846008800F03CFB641C684640888442E1DB03B030BD70B596480068002883
:20CC000004D12B48006A9449884201DAFCF770FA924E3468924D012C24DB08D12869401C36
:20CC20002861642803DA002000F0F7FA08E0002000F0E2FA002028618A48844200D10124F6
:20CC4000641C34608848844219DB64212000F9F773FC002803D0002000F0CEFA0FE000F080
:20CC6000DCFA0CE0002C0AD5002000F0D6FA3068401E30607D49884201D1FCF771FAFCF7CE
:20CC800096F97B49884228680AD37A4988420CDA002802D16868401C686028680A3005E0F9
:20CCA000002802D06868401C68600020286070BDB801002038B5704C2068401C20600A2899
:20CCC00011D16E480168491C01606D484168491C416000252560FFF78FFF6068401C606017
:20CCE0000A2800D1656000F06DFAFCF760F965490A68904200D802000A604A68824200D24B
:20CD000002004A6031BD0000102700004C1B002072B6002000F092FAFAE780B5FFF7F8FFF4
:20CD200001BD80B500F02AFA0220F9F7D2FD00F029FA01BD80B500F029FA0220F9F7C9FD1A
:20CD400000F028FA01BD704780B500F087F900F0B9F9F9F750FF01BD80B5CD20FFF73BF9BC
:20CD600001BD80B5CE20FFF736F901BD80B5CF20FFF731F901BD80B54348012141704348CF
:20CD8000F9F77CFF4248F9F742FF01BD10B584B00124E44310216846F9F74EFF009880280E
:20CDA00004D20199FCF742FA04001FE0C021490088420DD28039884203D101983549086028
:20CDC00013E0491C884211D10198334908600CE0803188420AD27F39884207D168460089FE
:20CDE000FFF7DCFD0199FAF7BCFC00242000F9F70EFF04B010BD000070B504001B2C04D318
:20CE0000BA2C01D2FFF784FF61342406A00D00BF26A1085880472148006A00240025204E3D
:20CE200031000C311F4A8B1E1B88002B0CD00B68C31A934208DB2800FBF7DAFBE800401B8E
:20CE400080003018448170BD6D1C1C31042DEADB70BD0000B8120020C0D40100441200202A
:20CE6000D00A0020FFFFFF7FB30200000CFEFFFF4C040000005C2605E40A0020BC120020AC
:20CE800000010020C0120020521B002038120020104704003C12002040120020B801002074
:20CEA00048120020C0270900704700001BCD0008BDBF000823CD000835CD000809C2000808
:20CEC00033C8000855920008D1C100081BCD000869CA0008A5CB000847CD0008D1E100084D
:20CEE00077CD00088DCD00081BCD00081BCD00081BCD0008DBC40008B7C300081BCD00089B
:20CF00001BCD000879C500081BCD00081BCD00081BCD00081BCD00081BCD00081BCD00083B
:20CF20001BCD00081BCD00081BCD00081BCD000863C2000885C2000809C300086DC80008A4
:20CF40007375000835760008F9740008F9C7000849CD000875D00008A5D000086DD00008C4
:20CF60009DD0000859CD000863CD00086DCD00081BCD00081BCD00081BCD00081BCD0008D4
:20CF800097C300081BCD00081BCD00081BCD00081BCD00081BCD000865D0000895D00008D5
:20CFA0005DC8000865C800087DD1000885D100081BCD0008C7A200081BCD00081BCD00081A
:20CFC0001BCD000837750008A3C3000879C4000821C2000809C9000855C900087BD40008B8
:20CFE0001BCD000831C200081BCD000811C1000879C200081BCD00088BC400086DC50008B8
:20D000001BCD00081BCD00081BCD00081BCD00081BCD00081BCD00081BCD00081BCD000890
:20D020001BCD00081BCD000859C300081BCD000880B5FCF767F8002002BD80B5FCF727F84F
:20D04000002002BD80B5FCF71FF802BD80B5FBF7DCFF01BD80B5FBF7EAFF01BD80B5FCF73D
:20D060000DF801BD80B5FBF7F9FF01BD80B5FBF7F3FF01BD80B5FBF7DEFF01BD80B5FBF750
:20D08000D9FF01BD80B5FBF7C9FF01BD80B5FBF7CFFF01BD80B5FBF7E6FF01BD80B5FBF7A9
:20D0A000DCFF01BD80B5FBF7CBFF01BD80B5FBF7C0FF01BD80B5FBF794FF02BD80B5FBF7E4
:20D0C0007DFF02BD80B5FBF77EFF02BD80B5FBF77CFFC0B202BD80B5FBF76BFF02BD80B55A
:20D0E000FBF778FF02BD80B5FBF779FF02BDFEE7F0B491B0030010000F226C463C34160064
:20D100000425F707FF0F7608002F02D037000F4E7E406D1EF5D12660521E241F002AEED592
:20D120001A7842405B1C1007800E6C462458100960400207920E6C46A25800095040491E83
:20D14000EED111B0F0BC7047000000002083B8ED70B50400074D28780600012803D1012C57
:20D1600001D000F017FA04492000FFF761FF2C70300070BD5B1B002040420F0080B5FFF7CF
:20D1800069FF01BD80B5FFF781FF01BD80B5FFF75DFF01BD80B5FFF775FF01BD80B58100A8
:20D1A00009184900414A51180A78002A01D0897800E04978002902D0FBF7F9FF01BDFBF75D
:20D1C000FFFF01BD70B50024384DAE88002E0FD0761E012E0BDAA878002801D02E8900E02A
:20D1E000EE8801214140A9702000FFF7D7FFAE800A3D641EE9D570BD012800DB704780B53F
:20D20000810009184900294A511801224A700978002901D1FBF7CBFF01BD012800DB7047B9
:20D2200080B5810009184900204A511800224A700978002901D1FBF7C3FF01BD012800DB2D
:20D24000704780B5810009184900184A51184A78012353404B700978002901D1FFF79EFFE9
:20D2600001BD012800DB704710B58200121852000E4B9A180B8813708B88D380CB88138104
:20D28000CB88002B08D08C88002C01D1002304E04C88002C01D0230001249380947009885E
:20D2A000002900D19180FFF779FF10BD200B00207047FEE7F1B584B00026BD4C2068002888
:20D2C00006D101960296082101A8F9F767FC5AE003A9684600F0EBF90098A168451A05D1E5
:20D2E0000398002805D1E568012602E001D5E0682D180498854200DA049501960498029041
:20D30000082101A8F9F74AFC0498002839D0A068009A90421FD36268151A04998D4200DD90
:20D320000D002E0013D03100F9F75FFCF9F7C6FC371AFBD0A068C019A0606168884201D33D
:20D340002068A060A06800F0BAF9F61BEED10498401B049015D0049D2900A068F9F745FC57
:20D36000F9F7ACFC2E1AFBD0A0688019A0606168884201D32068A060A06800F0A0F9AD1B19
:20D38000EED1F9F753FC05B0F0BD38B5884C05E06846017820001430FAF71CFD0121684622
:20D3A000FAF718FD6846007800282FD1606900F0ABF9050069682868F9F7C4F8A1698842D6
:20D3C00000D90800A061A9682868F9F7BBF8A169814200D20100A1612068002807D0E168B5
:20D3E000226991423BD0FAF7EFFD002020602069002829D16F4DFAF7B2FD40190540802002
:20D40000800085421FDA0020C04333E0012100A8401CFAF7DFFC684640780128B8D0022863
:20D4200002D0042805D009E06846017820001830B2E76846017820001030ADE768460078C7
:20D44000F9F704FCAAE725612069FAF797FD20602069E060216808186060002909D000F013
:20D4600016F923692268A169606900F0C0F82068A0600020F9F7CBFB31BD10B588B00121A1
:20D4800000A8801CFAF7A6FC68468078662820D10020019002E001A8FAF79CFC01216846FB
:20D4A000FAF798FC68460078002804D10198FFF701FF08B010BD012100A8401CFAF78AFC13
:20D4C0006846017840780328E5D00800F9F7BEFBE4E768468078642804D065280ED06E280A
:20D4E00023D0E6E7FFF751FFE3E7012100A8401CFAF770FC68460078F9F7A8FB0121684650
:20D50000FAF768FC684600780028EED1284C2068002806D000F0BBF82068FAF755FD002021
:20D5200020600020F9F773FBC3E70020019002E001A8FAF74FFC01216846FAF74BFC684615
:20D540000078002818D10198002802D00020C043E8E71C20F9F767FB0198F9F764FB002027
:20D5600000F0D2F80100142202A8FAF7DBFF142102A8F9F713FB9CE7012100A8401CFAF7CE
:20D5800029FC6846017840780128D1D00800F9F75DFBD0E710B5064C2068002806D000F029
:20D5A00076F82068FAF710FD0020206010BD0000B402002000FEFFFF474801890F22036883
:20D5C000134001D04260704744484269002A0DD0026911700169491C02684368D3189942FA
:20D5E00000D1110001614169491E4161704770B53A488161026043603949802464024A69B0
:20D6000022434A610A68630013430B60354D00262E6001680161416841618660C660816922
:20D620004808314A8018FDF73FF8082801D2082002E0A04200D3601E9021C9058A68C023C8
:20D6400013438B600A68C0239A430A600A68802313430B600A6A254B13400B620A6A2309D3
:20D6600013430B626E60AE60214A02400007400F1043A8811F4828601F480168FF229143D8
:20D6800040220A4302601D482103016070BD15480168242291430160194801688022920221
:20D6A0000A4302600168174A0A400260704772B60A4A53690B601169016062B6704772B619
:20D6C00006490A69824201D2801A02E04B689A1A1018486162B670471C440040F40A0020B0
:20D6E0001C1002400044004000D8B805FF0FFFFFF0FF0000258000001CE400E000E100E062
:20D7000010100240FFFFFDFF00A07047006CDC02C0000000FFFF000000000000000000004E
:20D72000016800E0491C0A78202AFBD0092AF9D00D2AF7D00A2AF5D001607047F8B50400E8
:20D740000F0000260025FFF7EBFF206801786A46437813701A020A43BB4B9A4234D1801CB4
:20D7600001780A00303AD2B20A2A01D230390CE00A00413AD2B2062A01D2373905E00A0071
:20D78000613AD2B2062A3ED2573900293BD4401C2A01551801780A00303AD2B20A2A01D2F6
:20D7A00030390EE00A00413AD2B2062A01D2373907E00A00613AD2B2062A01D320601AE008
:20D7C00057390029E3D5F9E72D2917D10126401C69460978401CAA0052195200303955186E
:20D7E00001780A00303AD2B20A2AF3D32060002E01D0280045423D600020F2BD0A00303AB0
:20D80000D2B20A2AE6D30020C043F2BD8F48006A704780B501000868496800916B46002212
:20D820000421FAF75BFF002802D50020C04302BD002002BD80B501000868496800916B461F
:20D8400000220221FAF74AFF002802D50020C04302BD002002BD80B50100086849680091A1
:20D860006B4600220121FAF739FF002802D50020C04302BD002002BD80B56B46002204219D
:20D880000068FAF71CFF002802D50020C04302BD009802BD80B5FAF72DFF02BD80B5FAF7A5
:20D8A00030FF02BD80B56B46002202210068FAF706FF002802D50020C04302BD009802BDB9
:20D8C00080B56B46002201210068FAF7F8FE002802D50020C04302BD009802BD10B5416829
:20D8E0000068401E1B2869D801A2125C974400BF1C242C343CCCCC445262728292CCCCCCDD
:20D90000CCCCCCCCCCCCCCCCCCCCA2C2080000F07AFF53E0080000F079FF4FE0080000F070
:20D9200078FF4BE0080000F077FF47E0080000F07BFF43E0FA20800041430800FFF77DFB87
:20D940003CE0002902D0FFF79DFB37E0FFF77EFB34E0002902D0FFF7A9FB2FE0FFF78EFB65
:20D960002CE0002902D0FFF795FB27E0FFF77AFB24E0002902D0FFF795FB1FE0FFF77AFBB9
:20D980001CE0002902D0FFF789FB17E0FFF76EFB14E0002904D0002000F04FFF102005E05C
:20D9A0000024E443200000F048FF200000F04AFF04E0481E8041C00F85490870002010BD5F
:20D9C00080B50168491E1B293BD801A2525C97441A20262C3238703E4C52585E6470707013
:20D9E00070707070706A70707072727200F0F9FE02BD00F0F9FE02BD00F0F9FE02BD00F005
:20DA0000F9FE02BD00F0F9FE02BD00F0F9FE02BDFFF718FBFA218900FCF746FE02BDFFF76B
:20DA20005EFB02BDFFF75FFB02BDFFF747FB02BDFFF751FB02BDFFF745FB02BDB948007859
:20DA400002BD002002BD000030780000B8010020F0B583B000680190081800906846FFF782
:20DA60005FFE02E00098401C00900098017800295FD0401C0A00613AD2B21A2A06D30A00CE
:20DA8000413AD2B21A2A01D35F294FD1012601E0761C401C01780A00303AD2B20A2AF7D362
:20DAA0000A00613AD2B21A2AF2D30A00413AD2B21A2AEDD35F29EBD0002E37D02AA50027B9
:20DAC00006246868B04208D1320000992868F8F7FBFC002801D1012702E00C35641EF0D1B8
:20DAE0000098801900906846FFF71AFE009800783D281BD10098401C009001A96846FFF776
:20DB00001DFE002F04D0A968080001D0019888476846FFF705FE00980078002809D068462F
:20DB2000FFF7FEFD009800783B289BD00020C04317E07C48007800280ED100BF1CA200BF7D
:20DB40001EA1482000F084FD062200211F2000F057FD00F033FD03E0012801D1F8F7F8FA82
:20DB6000002003B0F0BD0000F4F800080500000007E80008FCF80008050000000DE8000837
:20DB800004F900080600000013E800080CF900080600000019E8000814F900080B0000003B
:20DBA00029E8000820F900080E00000000000000000000000000000000000000FFFFFFFF21
:20DBC000FFFFFF3CE7000000B6487047B54870475C1B002080B500F038FE002002BD0020CB
:20DBE000704780B5006800F06FFD02BD80B5016800914168684600F07AFD02BD80B500686D
:20DC000000F0BEFC00F0DAFC002002BD80B5006800F0B6FC002002BD80B50068F8F759FEB4
:20DC200002BDF8B547688468C5680669006800F0EAFD380000F0EAFD200000F0EAFD2800D4
:20DC400000F0EAFD300000F0EFFD0020F2BD10B5006800F039FD10E010B582B001680091DE
:20DC60004168684600F043FD14E080B5006800F0A9FC02BD10B500F040FD040000F09EFCB8
:20DC8000200010BD10B582B0016800914168684600F048FD040000F091FC200016BD10B5E1
:20DCA00082B0016800914168684600F050FDF1E780B5FFF7CBF902BD80B5FFF7E3F902BD58
:20DCC00080B50068FFF744FA02BD10B50C00C368816862184168611800682018FBF7EEF9BA
:20DCE00010BD0020C043704780B50A00416800681018F8F7A1FF02BD80B50A004168006867
:20DD00001018F8F74BFF02BD80B50068FFF795F902BD80B50068FBF7EFF802BD8E48006A8E
:20DD2000704700005B1B002080B50068002802D0FFF7B0F902BDFFF795F902BD80B50068C1
:20DD4000002802D0FFF7AEF902BDFFF793F902BD80B50068002802D0FFF7A0F902BDFFF751
:20DD600085F902BD78B402688A1843688168C068DC0812195B075B0FFF25FF249C40C0189C
:20DD8000083803D54642354125402C001578A5430E009E4034402C431470012801DA0020F0
:20DDA00013E0521CD940082807DB08381170521C090A0828F9DA002807D001248440641E28
:20DDC0001078A0430C400443147072BC704738B50268D2B245688368CC1891490978002901
:20DDE00012D001290ED12D0607D0002104201043F8F754F92100032001E021001000F8F715
:20DE00004DF932BD0120C04332BD10B501000868C0B24B688968824C2478002C0CD0012CCF
:20DE200008D11B0602D0042202431000F8F7E8F8020001E00122D243100010BD80B5006837
:20DE4000C0B2072805D28000764908588047FF2801D10020C04302BD1248704711487047E8
:20DE6000104870470F48704780B50068FDF70CFB002002BD80B5FDF746FB002002BD80B590
:20DE80000A00416800681018FDF790FB02BD80B50A00416800681018FDF749FB02BD014849
:20DEA00070470000FAFEFFFFF7B50600C800401A8000C44908188769002F01D1042037E008
:20DEC0003868C149884206D101220092BA68CD2A01D301202CE0884221D13C002034F8687C
:20DEE000C000381820300190002501E008346D1CF86885421BDA02992068019A1018F8F775
:20DF00003FFB0028F2D1646850213000F9F728FD45A0F064009800280CD038690AE0AB4906
:20DF20000298F8F72DFB002801D10424ECE70320C0430FE03818B0643464B06C0268F2634F
:20DF40000099002905D0121FF26304218018F8F79BFA002003B0F0BDB8010020F5B581B02F
:20DF6000C800401A8000974908188669002E01D1042039E00020009030689349884206D10E
:20DF800001220092B268CD2A01D301202CE0884221D134002034F068C00037182037002593
:20DFA00001E008346D1CF06885421CDA029920683818F8F7E5FA0028F3D1646850210198A3
:20DFC000F9F7CEFC019800BF17A1C164009800280CD030690AE07D490298F8F7D1FA0028F1
:20DFE00001D10424EAE70320C04316E0301801998864019804640198806C02680199CA63B5
:020000040800F2
:20E000000099002906D0121F0199CA6304218018F8F73AFA019800F069FD03B0F0BD000041
:20E020005B1B0020F8010020B9DC0008B1DC0008C1DC0008CBDC000809DD000813DD0008C5
:20E04000E3DC0008E9DC0008F9DC00081DDD000829DD00083DDD000851DD000865DD00089D
:20E060000BDE0008CFDD00083DDE00084FDC000859DC00086BDC000875DC000885DC000857
:20E080009FDC000823DC000857D8000835D8000813D80008C1D80008A5D8000879D8000838
:20E0A00095D800089DD80008DDD80008C1D90008DFDB0008DFDB0008E3DB0008EDDB0008F5
:20E0C000FDDB00080DDC0008D5DB0008DFDB0008DFDB000851DA000819DC0008DFDB000841
:20E0E000DFDB0008DFDB0008DFDB0008C9DB0008CDDB000859DE00085DDE000861DE0008B5
:20E1000065DE000869DE000875DE00087FDE00088FDE00089FDE0008F0B585B00F001600AC
:20E120000B2804D110216846F8F786FD06E00C216846001DF8F780FD002000900098C0B282
:20E14000009002982049884200D10398019945181C4C0098C100081A800020188069002853
:20E1600010D000F034FB0098C100081A800020188069F9F729FF0098C100081A8000201839
:20E180000021816128006030F9F7F8FE040010D0082269460831FAF7B1F901990839200052
:20E1A0000830F8F749FD2021601900F001FB3C6003E001980838F8F749FD0098306005B0E2
:20E1C000F0BD0000481200205043563264E3000830B5A3B0012104A8F8F72EFD6846007C64
:20E1E0000A2800D9B3E002A1095C49008F4400BF06080DAFAF406677AF8E9F00564801E0AD
:20E2000000F08EFCF8F703FDA1E06A4601A90220FFF782FF514C0098C100081A8000201851
:20E22000019981614B4D00BF4EA200992800FFF795FE0990286C0A9028680B90E86B0C90F0
:20E24000686C0D9000F0C3FA0098C100081A800020188069002808D0F9F7B6FE0098C10087
:20E26000081A8000201800218161142109A86CE0002500246A4601A90520FFF74DFF042061
:20E28000019900290AD00099CA00511A8900334A5118019A8A610290039502E00290E44359
:20E2A0000394082102A8F8F779FC002C4FD400BF2CA200212748FFF7F7FD48E0274C00257A
:20E2C000A069002805D000F082FAA069F9F77CFEA561042002900395082102A835E00821F4
:20E2E00005A8F8F7A9FC1B4D1D4B069A0599280000F062FD4C210E910F90482229000EA864
:20E300000830FAF70FF950210EA81EE00C2105A8F8F792FC042105A8001DF8F73FFC069998
:20E3200005980C4A926C1018F8F738FC0FE00C2105A8F8F781FC06990598064A926C1018BA
:20E34000F8F77AFC042105A8001DF8F727FC23B030BD0000B80B0020E6070000481200204D
:20E360000DD800086D61696E00000000FDB484B0914AD36ADC105807400F0090059D08201A
:20E38000009E801B854200DD05000126AE40761E506B00190290906B00190190300008406F
:20E3A0006F4638736846007C06400098002801980ED00078009FBE4006430198067002984F
:20E3C00000786E46367B009FBE400643029803E0067002986E46367B06700598401B5B19A6
:20E3E000002809D0641C6E46367C2E41976B3E552941556B29551B18D36207B0F0BC704708
:20E4000010B50400082C07DB0822FF21002000F0F7F8083C082CF7DA012C06DB0122012138
:20E42000002000F0EDF8641EF6E710BDF0B583B006000C00150060484088401B071B0422A9
:20E440000021032000F0DCF8002F0DD05A48016A0020C043814204D03A00002000F0D0F8CF
:20E4600002E03800FFF7CCFF5348C06A019008E00020009A3178C0B200F0C2F8761C0098DA
:20E48000241A012C0CDB0820082C00DC20000090002DEDD1092CEBDA0120611E8840E8E726
:20E4A000002D14D04448416A0020C043814204D02A0001206B1E984007E0022D02DB681E35
:20E4C000FFF79EFF01220121012000F099F801220021012000F094F8019803B0F0BD79B5BA
:20E4E00082B00C001D00561B761E03220021012000F086F8002E04D032000021002000F082
:20E500007FF82D48C06A00900AE00020320002990978C0B200F074F80298401C0290A41BE8
:20E52000012C0BDB0826082C00DC2600002DECD1092CEADA0120611E8840E7E7002D06D048
:20E540002A00002101206B1E984000F059F801220021012000F054F8009804B070BD10B5CE
:20E56000154CE36A002B0AD056480078012804D1226BA16B606BFAF7A1FD0020E06210BDB2
:20E5800010B5040006D001220021002000F038F8641EF8D110BD80B507480178002903D047
:20E5A0004168491C416001BDC16AC91D07229143C162FFF7D4FF01BD0801002080B5FFF7E2
:20E5C000CEFF01BD10B50400FFF7C9FFE0101F49096B091808784A7812020243887803049A
:20E5E0001343C87800061843091D6207520F06D0D040030008782021891A8840184310BDF7
:20E60000F8B506000D001400104F7878002808D0062200211F20FFF7A9FEFFF7BCFF0020E1
:20E620007870F86A009008E027003A00E9B2F0B2FFF79CFEE41B360A2D0A012C03DB092C34
:20E64000F2DB0827F1E70098F2BD000008010020F2B584B004001700C01DC6082ED0784D12
:20E66000A86AE96AC91DC910401A80218900884206D2FFF774FFA86AE96AC91DC910401A69
:20E68000864200D830000190E86A0290019D092C02D30820009000E00094009A397804987A
:20E6A0000078FFF763FE0498401C04907F1C0098241A6D1EEBD10198361AD0D1029805B06E
:20E6C000F0BD00005B1B002001B58148C169002900D001E0002002BD02696846FFF7A6FEE2
:20E6E00002BD7B4AD3689268FFF7F9FE02BD80B5002901D1002002BDF3E738B57448C56AF4
:20E700008168C0680C1A641E032200210120FFF777FF002C04D0220000210020FFF770FFA5
:20E72000280032BDF8B506000C006948C76A0AE00825082C00DC25002A0031780020FFF7EC
:20E740005FFF761C641B012CF2DA3800F2BD70B582B006000C005E48C06A009007E000209A
:20E760002A003178C0B2FFF74BFF761C641B5848C068012C0BDB0825082C00DC250000289E
:20E78000EDD1092CEBDA0120611E8840E8E7002807D0020000210123401E83401800FFF715
:20E7A0002FFF012200210120FFF72AFF009876BD474A1063431853634B00C01890639162BE
:20E7C0000020C043106250620020D06270474048816A002904D00021016341638163816289
:20E7E00070473B48806970473948406970473848006970473648C06870473548C069704704
:20E800003348408870473249886110E03049486105E02F49086109E00949C8604869CA687C
:20E820008018401C886070470549C86188690A698018CA69801848807047254908627047F9
:20E840000801002022494862704738B52048006A0021C943884235D0FAF716FC04001D4D97
:20E86000AC4204D1FFF797FE1B48FEF7E6FB062200211F20FFF7C4FE042200210320FFF771
:20E88000BFFE052210211020FFF7BAFE062200211F20FFF7B5FE042200210320FFF7B0FE46
:20E8A000052210211020FFF7ABFE022200210120FFF7A6FEAC420AD1FFF76DFE2800FEF7EA
:20E8C000BCFB31BD062200211F20FFF799FE31BD0801002018FCE70388130000012000BDF0
:20E8E000022000BD0A0B9200A3585B1EA35002D00A05120EB61AB95BB61CCA06520EA85844
:20E9000087460A0552160B0B9B00195989181951F1E70A05120F92000B0B9B00E3580906F0
:20E92000090F5918A150B95BB61CCA06520EA858874660B40E0BB600A65901E060B40E0B8A
:20E940000B051B0F9B00E5580906490F8900734808588746AD19E550002D03D101226264E8
:20E9600060BCC8E70022626460BCC4E7AD1BF2E73540F0E73543EEE77540ECE7B540EAE795
:20E98000F540E8E77543E6E70A0B92000905490EA150B0E70A0B9200B95BB61CBB5BB61CE5
:20E9A0001B040B43A350A6E7626CD20703D5A2E7626CD2079FD509040916490076189AE7C3
:20E9C000626CD207D20F090B8900625093E7CA09E36BF8184906490F8900C918E163390027
:20E9E000E36C9A5800F002F8206084E710478A0603D5E26B121FE263BE500904891549007D
:20EA0000761878E78A06F8D5E26B121FE263BE50090B890066586EE70A05130F9B00E31864
:20EA20000A0B9200E06B801A19003B18E06308681860091D1B1D121FF9D15CE70A05130FE6
:20EA40009B00E3180A0B9200E06B39188018EDE7E26BD659121D490989005218E2634AE70B
:20EA6000CA12D2065216E36BD2188B051B0F9B00490502D5E358D3513DE7D259E2503AE7C7
:20EA800020B44806420F0D052D0FAD00080B800020180368FB1809061CD5110003D118784A
:20EAA000605120BC27E7012A03D11888605120BC21E7022A03D11868605120BC1BE70178FF
:20EAC0004907490F0068C0083818F7F7B7FC605120BC10E76059110002D1187020BC0AE7F7
:20EAE000012A01D11880F9E71860F7E7F0B5A0B0040000AD266C07498022043A8B58AB5005
:20EB0000FBD100F003F8266420B0F0BD00B5A76CF1E6000014020020F7E8000894020020C5
:20EB2000CC207047016C891E016401207047016C891E0164022070470A0B920080180268E6
:20EB40000905491651180160002070470A0B9200821813685B1E136004D0026C0905090E98
:20EB6000511A01640020704718B40A06520F0B051C0F0B0BC90601D499004358A10041188E
:20EB80000C68002A01D1E31819E0012A01D1E31A15E0022A01D1234011E0032A01D123436B
:20EBA0000DE0042A01D1634009E0052A01D19C4004E0062A01D1DC4000E05C4323000B60F0
:20EBC0000021002B00D101214164002012BC70470A05120F92000B0B9B00C3580906090FF7
:20EBE00059188150002070470A0B92000905490E81500020704710B4026C836C9B181C88D0
:20EC00005B881B042343121D0264090B89004350002010BC70474422825CD20705D5026CBF
:20EC200009040916490051180164002070474422825CD20705D4026C090409164900511878
:20EC400001640020704709138900020044321278D307DB0F43500020704710B504000A00D0
:20EC6000E06B5106490F89004118E163A16C0818520A9200E36C9A5890472060002010BDD4
:20EC800018B48A0605D5C26B121FC263836C046C9C50026C89098905491551180164002096
:20ECA00012BC704718B48A0605D5C26B121FC263836C046C9C500913890041580164002008
:20ECC00012BC70470A0B9200C36B9B1AC3630905090F89004118806CC0180B680360091D37
:20ECE000001D121FF9D10020704718B40A0B92000905090F89004118C36B846CE4189B18DD
:20ED0000C36320680860241D091D121FF9D1002012BC704710B4C26B836C9B18C9081C2432
:20ED20000C40241D1119C16319680164002010BC704770B504004806420F0805050F080B73
:20ED400080002058A36C1E18090614D5002A01D130780DE0012A01D1308809E0022A01D151
:20ED6000306805E04107490FC0081818F7F766FBA90060500AE0A8002058002A01D1307030
:20ED800004E0012A01D1308000E03060002070BDCA12D2065216C36BD218836C9A188B05C0
:20EDA0001B0F9B00C018490502D50068106001E01168016000207047F4B5A2B006000C001A
:20EDC0001F00802212A101A8F9F7ACFBB06C00902298002802D0B84722994518306C0099D3
:20EDE000095A801C30643000CA06520E01AB9A58904700280AD1002C01D0641E05D022989A
:20EE00000028EBD0B847281AE8D1002023B0F0BD25EB000869EB00082FEC00085BEC00088F
:20EE200081EC0008D1EB0008E9EB0008C5EC000833ED000839EB00084DEB000815ED000866
:20EE400091ED000847EC00082FEB00082FEB000825EB000869EB000817EC00085BEC0008DF
:20EE6000A5EC0008D1EB0008F7EB0008EBEC000833ED00082FEB00082FEB00082FEB0008DE
:20EE80002FEB00082FEB00082FEB00082FEB000878B4C300534C002A246804D0E318524C39
:20EEA0001B19198012E0E318504C1B19002501263F2902D24C080E4002E04C090125E1065A
:20EEC00000D0641CE903A4020C431C80400080188000BE490B5071BC70478000A54A101830
:20EEE000C0229201036813408B4200D1704730B482B000910368009C634000939E4B009C21
:20EF00001C430094BD4C14E080009A4A10183022036813408B4200D1704730B482B0009169
:20EF20000368009C63400093934B009C1C430094AC4C009D25400095009D056005682A40BF
:20EF40008A420CD000910168009A5140009100990B43009300990C4000940099016033BC77
:20EF6000704710B584B083480168A54A0A4002609648006800888205920D080518D5A1483B
:20EF8000006802A9022A06D303880B80801C891C921E022AF8D2002A01D00088087002A8B7
:20EFA000FCF77AF8C02189010020FFF796FF16E0002A14D01000934909686B46022808D3BF
:20EFC0000C881C80891C9B1C801E0228F8D2002801D00888187069460020FAF7C5FD04B0CC
:20EFE00010BD0000505C00400260004006600040F8B5604C606C9E21090201404A053AD582
:20F00000AB4860649C200002206400202065AC4D402129617B4F39006C4A2023086010609A
:20F02000121D091D5B1EF9D1286929690A312961216DA44A89180880A34E088880193860F9
:20F04000002208210020FFF723FF286929690A312961216D89190880088880197860012269
:20F0600008210020FFF714FF984820608020E064FAF7EFFEF1BDCA0411D595486064A16C0C
:20F08000C02000020840E10B88420CD000286FD0206C0C2188432064FAF7FDFEF1BD0A059C
:20F0A0000CD58C486064FAF7EEFE206C082101432164206C042101432164F1BD0A0451D520
:20F0C0000607360FC106C80F002E0AD1002802D0FFF747FFF1BD2068A04901402160002000
:20F0E0003DE0B10061180028086834D0444A02400A60610C3000FFF7F0FEF100334840586E
:20F1000000888205920D412A01D3402201E0002A17D010003B4B5958694D2B001433022815
:20F1200008D30C881C80891C9B1C801E0228F8D2002801D008881870143529003000FAF732
:20F1400013FD5F48805D002812D0C02189013000FFF7C3FEF1BD814A02400A603000FAF779
:20F16000FAFDF1BD880501D5A74800E0A7486064F1BD0000005C00408080000038B50500C9
:20F180000C00002D16D0FAF7A6FA000608D5002C01D0102100E020212800FFF7B5FE31BDCE
:20F1A000002C02D08021490101E0802189012800FFF793FE31BD80B595490020FFF7A4FEF2
:20F1C00001BD80210143934801607047480D002010B5040080218901FFF77FFE8E480021C6
:20F1E000015510BDBF8FFFFF10B50400C0218901FFF773FE88480121015510BD8FBFFFFFA4
:20F200008F0F0000C80C0020F8B58448B830009040688047824C03202064012020640026BC
:20F220006664800220647F480099096888479C20000220642665224D40202861264F38008C
:20F240007949202206600E60091D001D521EF9D1286929690A312961216D1A4A8918088056
:20F26000194E088880193860002208210020FFF70FFE286929690A312961216D8919088058
:20F28000088880197860012208210020FFF700FE0E4820608020E064FAF7DBFD009880680A
:20F2A0008047F1BD80B55D48EC300068804701BDFFFBFFFF5D490878401C0870C0B27047DB
:20F2C000C80D0020046000400060004030320000FFEFFFFFFFF7FFFFC80C002070B54279DF
:20F2E00053065B0E0188D20900240079002804D0012805D0032805D006E08024A40003E040
:20F30000802400E0C024E400002A01D0202001E080208001204318439C00414D28513E4D78
:20F320002C692E69881C30182861DD004048414E002A366802D075192D1802E075193E4ECF
:20F34000AD192C805C00A418A4003C4E2D88281830511800FFF79CFD70BD00000F8F00000D
:20F360007047002801D04020704708207047F5B581B00C00C7003148C01945681646E007F7
:20F380000BD5022A12D32000FAF76BFE2880AD1CA41CB61E022EF6D208E0022E06D320886C
:20F3A0002880A41CAD1CB61E022EF8D2002E01D0207828801C48C0194068029901803021BD
:20F3C0000198FFF7A1FD03B0F0BD80B5FAF742FC01BD80B52021FFF797FD01BD00207047E9
:20F3E00010B50400FAF777F9A1000D4A51180A68000601D5402001E08020C001024201D07D
:20F400001043086010BD0000FFFDFFFFFF61FFFF101000004C5C0040C80D00206C0F002074
:20F42000005C0040F1EF0008480D00205A1B002000600040505C004004600040C80C00201A
:20F44000FEE7000030B483B05048016801220A43026041684E4A0A40426001684D4A0A4066
:20F46000026001684C4A0A40026041684B4A0A404260C16A0F229143C162016B484A0A40BA
:20F480000263416B0122914341630021816001910091110402680A430260A023DB014A0084
:20F4A000046814400094019C641C0194009C002C02D1019C9C42F3D103689B03DC0F0094E4
:20F4C000384B1124009D012D1C6023D141684160416841604168344A0A40426041682204C3
:20F4E0000A4342600168802252040A4302608021890402680A40FCD041680322914341601C
:20F50000416802220A4342600C2142680A40082AFBD10CE0436B19434163416B1140FCD0AD
:20F52000416803229143416041680A43426003B030BC704730B51D4C20680C210140082925
:20F5400002D00C2916D017E0206822680F21850C0D40AD1CC0204002104003D114484543B4
:20F5600028000AE0A26A13481140491CFBF79CF8684302E0104800E00E481049086122686F
:20F580001206120F8A5CD040086130BD001002400CB8FF08FFFFF6FEFFFFFBFFFFFFC0FF22
:20F5A000ACFEFFFF00200240FF7FC0FF0410024000093D0000127A00006CDC02200300204F
:20F5C000F0B586B00200083201688900511800914068C107C90F0591012188438000009944
:20F5E00008180490002400210026002301200290019003E00027019785421AD10098049DF8
:20F60000A84202D1284606B0F0BD0568001D03900598002801D048462D1803980068281893
:20F62000039F3F1D0097E7E7116854185168611808328C42F8D0029F002F0ED0267876B20C
:20F64000641C002702970127019704E0116854185168611808328C42F8D0002E14D5019F28
:20F66000002F01D02378641C8542C3D02B706D1C761C0BD5F8E78542BED08C42BCD0237856
:20F68000641C2B706D1C761E002EF4D501270297B2E7FEE782B0F9F79BFD234A811A491CD5
:20F6A0001000F8F7AFFCF9F76DFCFDF701FE0020FDF7A2FDF9F79EFC1C48FDF7BEFCF9F715
:20F6C00076FC0120FCF786FCF7F7FEFAFDF7ECFBFBF728F80027FF43154C164D012604E017
:20F6E000FDF7ACFD3220F7F7F4F8F7F706FB0028F6D0114806600020FDF77EFD0EE02660A2
:20F700006846F7F7FEFA002808D42760FAF7FFFF68460078FDF770FBFAF7F4FF28780028AA
:20F72000EDD0F7F7E1FAE0E7601D0020204E0000441200205D1B0020B812002010B5254C43
:20F740002078401C2070F9F731FDFDF7B3FA00F049F872B62078012804D16068002801D0B6
:20F76000F8F781F92078401E207062B610BD38B572B6184C6078401C6070FFF7DBFE16480B
:20F780000068FA218900FAF78FFF8021490488421DD2124A491E0840401E5060104803685B
:20F7A0000B40C0252D061D430560002393600723136002681140802212060A430260607872
:20F7C000401E60706078002800D162B631BDFEE730BFFDE7B80100203003002010E000E070
:20F7E00020ED00E038B5154B1A1D2833D868002803D001201874507017E0D469641CD461AC
:20F8000003CB083B0025401C694103C3083B106A201A01D401205070187A002805D0401E4C
:20F820001872000601D1012010700548046802E0606880472468002CFAD131BDB801002051
:20F840008C0B002000B583B072B60F484178491C4170FBF75BF8F7F728F8FFF788FF0B4898
:20F8600002210291C021C90001910090084B032209A154020019FCF783F906480121017025
:20F88000F8F7D3F803B000BDB80100200815002095F60008561B00204A2D4C696E6B0000FF
:20F8A00009F20008B5F20008DDF2000861F30008A5F2000863F30008DDF30008C3F10008D2
:20F8C0007DF10008B7F10008D1F10008E9F10008CBF300086FF30008D3F30008E1F300087C
:20F8E0000000000000000000000000000000000000000000495250726500000044525072EE
:20F90000650000004952506F737400004452506F7374000049524C656E44657669636500FB
:20F92000506572666F726D544946496E6974000053454747455200004A2D4C696E6B0000B3
:20F94000317E00083B7E0008D57D0008157E00084B7C0008437D00086D7D00085D7C0008D0
:20F96000FF7C0008797E000810B5074979441831064C7C44163404E0081D0A6889188847A3
:20F980000100A142F8D110BD08000000380000004F6AFFFF60150000000600200400000057
:20F9A000601D00200000000019FCFFFF0200000002000000B20000000604000008010020AE
:20F9C000F6040000080C10141820303100040C1014181C24282C3034FFFFFF3839000000AA
:20F9E00000F009F8002801D0FFF7BEFF0020FFF729FF00F002F80120704780B500F002F84B
:20FA000001BDFEE70746384600F002F8FBE7FEE701491820ABBEFBE72600020001488047C2
:20FA20000148004745F400082DFA0008C046C046C046C046FFF7D4FFF1A000000000000054
:20FA4000FEE7FEE7FEE7FEE7FEE7FEE7FEE7FEE7FEE7FEE7FEE7FEE7FEE7FEE7FEE7FEE756
:20FA6000FEE7FEE7FEE7F8000001E900F8FFEC0003B80B0000FA3005313233343536FC00EC
:20FA80000F6613010130F9000838F90008480100208B000040E6007EE7D00008C5D000087E
:20FAA000D7D00008BDD00008B5D00008CDD00008DFD00008DDE8000833E90008A9E900088E
:20FAC000CFE90008EFE9000813E9000889E9000819EA000881EA000803E90008E5E80008C1
:20FAE00051EA000861EA0008C1E90008E1E80008E1E80008DDE800083DE90008B1E900087F
:20FB0000CFE9000805EA000813E9000895E900083DEA000881EA003C08E1E80008E1E8002C
:20FB200008E1E80008E1E80008E1E80008E1E80008E1E8000855E900086DE9000871E900AA
:20FB40000875E9000879E900087DE9000881E9000885E90008EF000010FA000C80250000CD
:20FB6000A58D95BD87AFB79FFFFB000B010081A9B199A38B93BBFFE0FBFF0000F7FF00E0D0
:20FB8000FCFFEA000889BA0008B1BA000832F5007E0102030406070809006CDC0208B402E5
:20FBA0004B9C4608BC6047C0461BD2000808B4024B9C4608BC6047C046F9D1000808B402C6
:20FBC0004B9C4608BC6047C046E3A800089748984901607047F8B40023944C994D25600002
:20FBE00026F6430700001D3F68B74201D0002008E05B1CA70DBB4201D125600023091FF04F
:20FC0000D10120F2BC7047F7B584B0EFF31080027E9072B6002001908B480068C0070BD471
:20FC2000894800680121014387480160864800688007FBD5012001907F4C002B49D004980B
:20FC40007E4901400202120A914242D17C4F06994118491EC90A39400091C00A0740B94283
:20FC600037D3F802802109054618704DE068000603D575482060754820600020E060A069AD
:20FC8000400705D473482860062068607248A8607EE10C3000FFF79FFF002814D10220E013
:20FCA000602661E06840210143E160FFF790FFA068C107FAD4E16802229143E16014210154
:20FCC0004001D01420A0607F1CE00C36180098B842CCD2069840100599049AE3681B060341
:20FCE000D55A4B23605A4B23600023E360A3695B0706D44E4D574B2B6006236B60564BAB29
:20FD0000600123E3604B4B494D0E88534FBE42117ED01788B74200D01680921C891C2B607D
:20FD2000A668F707FBD41427374006D0A06814210143A16003E0921C891C401EE5D1012073
:20FD4000C043E1680140E1600199012904D13E49096808403C490860029880F31088069ACA
:20FD600005990498FFF72CFF002804D107B0F0BD0020FFF715FF06984400012CF8DB00209B
:20FD8000FFF716FF641EFAD1F2E7F0B583B0EFF37E1081019172B60021002601272A4C22A8
:20FDA000683A4007D122683A432260022223681340FCD00126214A0240F806101800901E8A
:20FDC0004DE868000603D52148286021482860E960A869400706D416481E490160062141BD
:20FDE000601D498160E10C0098FFF7F6FE002814D10220E86000982861E86840210143E977
:20FE000060FFF7E6FEA8683842FAD1E9680222911E43E9601421084000D0A960012E02D14B
:20FE20002068B8432060019880F3108803B0F0BDFD0014300040AAAA00000420024000F888
:20FE4000FF00FF1F0000AAAAFD002010024023016745AB89EFCD55550000FF0F0000FFFF4C
:20FE600000000B214843401EFDD57047FFFFFFFFFFFFFFFFFFFFFFFFFFFFFFFFFFFFFFFFF8
:20FE8000FFFFFFFFFFFFFFFFFFFFFFFFFFFFFFFFFFFFFFFFFFFFFFFFFFFFFFFFFFFFFFFF82
:20FEA000FFFFFFFFFFFFFFFFFFFFFFFFFFFFFFFFFFFFFFFFFFFFFFFFFFFFFFFFFFFFFFFF62
:20FEC000FFFFFFFFFFFFFFFFFFFFFFFFFFFFFFFFFFFFFFFFFFFFFFFFFFFFFFFFFFFFFFFF42
:20FEE000FFFFFFFFFFFFFFFFFFFFFFFFFFFFFFFFFFFFFFFFFFFFFFFFFFFFFFFFFFFFFFFF22
:20FF00007777772E7365676765722E636F6D00436F70797269676874202863292032303025
:20FF200033202D203230313220534547474552204D6963726F636F6E74726F6C6C65722EF3
:20FF4000204D6179206265207573656420696E206F726967696E616C204A2D4C696E6B739E
:20FF600020616E642070726F6475637473206D616E75666163747572656420756E6465723D
:20FF8000206C6963656E7365206F6E6C792E00FFFFFFFFFFFFFFFFFFFFFFFFFFFFFFFFFF5F
:20FFA000FFFFFFFFFFFFFFFFFFFFFFFFFFFFFFFFFFFFFFFFFFFFFFFFFFFFFFFFFFFFFFFF61
:20FFC000FFFFFFFFFFFFFFFFFFFFFFFFFFFFFFFFFFFFFFFFFFFFFFFFFFFFFFFFFFFFFFFF41
:20FFE000FFFFFFFFFFFFFFFFFFFFFFFFFFFFFFFFFFFFFFFFFFFFFFFFFFFFFFFFFFFF3ADA0B
:00000001FF
